:100000009EC10000CDC10000CBC10000C9C10000ED
:10001000C7C10000C5C10000C3C10000C1C10000CC
:10002000BFC10000BDC10000BBC10000B9C10000DC
:10003000B7C10000B5C10000B3C10000B1C10000EC
:10004000AFC100000C94B03FABC10000A9C10000DB
:100050000C94DE3FA5C10000A3C100000C94DC3E5F
:100060009FC100000C94A63E0C947C3E99C10000F8
:1000700097C1000095C1000093C1000091C100002C
:100080000C94823F8DC100008BC1000089C100002B
:1000900087C1000085C1000083C1000081C100004C
:1000A0007FC100007DC100000C94543F79C1000065
:1000B00077C1000075C1000073C100000C94263F99
:1000C0006FC100006DC100006BC1000069C100007C
:1000D00067C1000065C1000063C1000061C100008C
:1000E0005FC100004E414E494E495459494E46CDDC
:1000F000CCCC3D0AD7233C17B7D13877CC2B3295DF
:1001000095E6241FB14F0A000020410000C84200BC
:10011000401C4620BCBE4CCA1B0E5AAEC59D740086
:10012000407A10F35A00A0724E18090010A5D4E8C6
:100130000000E87648170000E40B54020000CA9A59
:100140003B000000E1F505000080969800000040AB
:10015000420F000000A086010000001027000000F0
:1001600000E803000000006400000000000A000036
:100170000000000100000000002C76D888DC674FEA
:100180000823DFC1DFAE59E1B1B796E5E3E453C61A
:100190003AE651997696E8E6C28426EB898C9B6212
:1001A000ED407C6FFCEFBC9C9F40F2BAA56FA5F4BC
:1001B00090055A2AF75C936B6CF9676DC11BFCE0E4
:1001C000E40D47FEF520E6B500D0ED902E03009437
:1001D0003577050080841E080000204E0A000000CC
:1001E000C80C333333330F986E12831141EF8D21D6
:1001F00014893BE65516CFFEE6DB18D1844B381B3D
:10020000F77C1D901DA4BBE424203284725E228101
:1002100000C9F124ECA1E53D2700002200250028BB
:10022000002B002E003100340002010000050108FF
:10023000010B01000020002300260029002C002FC4
:100240000032000001000003010601090100000A5C
:100250000B02090C0D0E080703040100000000004A
:10026000000000000000000000000000000000008E
:10027000000000000000000000121110000000004B
:10028000000000000000000000000000000000006E
:1002900000000000002100240027002A002D00306B
:1002A00000330001010000040107010A01010210EE
:1002B0002020080810204010204080020102010880
:1002C0000402010102040810204080804020100830
:1002D0000402018004020180402010080402010889
:1002E00004020101020408102040800102040810E9
:1002F00020408005050505070508080808020202D8
:10030000020A0A08080404040401010101010101B0
:10031000010303030303030303040707070C0C0C87
:100320000C0C0C0C0C02020202060606060606065F
:10033000060B0B0B0B0B0B0B0B0028409D4D1124D8
:100340001FBECFEFD1E2DEBFCDBF00E00CBF18E093
:10035000A0E0B2E0E8EEF0EB00E00BBF02C00790D7
:100360000D92A231B107D9F724E1A2E1B8E001C0B2
:100370001D92A531B207E1F711E0CEE9D1E000E02E
:1003800006C021970109802FFE010E946357CD39D5
:10039000D10780E00807A9F70E9419420C9463581E
:1003A0002FCE883591050CF04BC085359105CCF4E6
:1003B000803391054CF58D3291059CF48C3191057B
:1003C000BCF4893191056CF48E30910564F48B3066
:1003D00091053CF4009729F097FD08C00297049717
:1003E00028F481E008950F970997D8F380E00895E5
:1003F000863291053CF4843291059CF74F97039720
:10040000A8F7EFCF8997FBCF843491056CF4813442
:1004100091053CF78A3391052CF4873391050CF74D
:10042000C397EDCFCD97EBCF8E34910534F48B3459
:100430009105BCF687549109E2CF81559109DFCF30
:10044000863891051CF5833891055CF68237910555
:1004500084F48F3691052CF6883691053CF4853668
:1004600091050CF0BECF8B559109C9CF89569109E2
:10047000C6CF8C3791053CF4893791050CF0B1CF8C
:1004800083579109BCCF8D579109B9CF803D910514
:100490008CF48D3C91050CF0A4CF843991053CF48B
:1004A000813991050CF09DCF8D589109A8CF895CB9
:1004B0009109A5CF8A3D91053CF4873D91050CF04B
:1004C00090CF835D91099BCF8D5D910998CF9C0161
:1004D000803E910508F021C5FC018827ED58FD4FAD
:1004E0008F4F0C94635753036003690372037F03B8
:1004F00088038D078D078D078D078D079503A20350
:10050000AF038D07BC03C503CE03DB03E403ED0398
:10051000F603FF0308048D0711041A0423048D0752
:100520008D078D072C0435043E048D078D07470485
:1005300054048D078D078D0761046E047B048D07BD
:10054000880491049A048D078D078D07A304AC04D9
:10055000B5048D07C204CF04DC048D078D078D0719
:10056000E904F60403058D0710051D052A058D070E
:100570008D078D073705440551058D075E05670515
:1005800070058D078D078D079405A105AE058D07B4
:10059000BB05C805D5058D078D078D07E205EB0561
:1005A000F4058D078D078D078D078D078D078D0746
:1005B000FD0506060F068D07180621062A068D077B
:1005C0008D078D07330640064D068D075A066706D0
:1005D00074068D078D078D0781068E069B068D0795
:1005E000A806B106BA068D078D078D07C306CC068F
:1005F000D5068D078D078D078D078D078D078D0714
:100600008D078D078D078D07790582058B058D0771
:100610008D078D078D078D078D078D078D078D073A
:100620008D078D078D078D078D078D078D078D072A
:100630008D078D078D078D078D078D078D078D071A
:100640008D078D078D078D078D078D078D078D070A
:100650008D078D078D078D078D078D078D078D07FA
:100660008D078D078D078D078D078D078D078D07EA
:100670008D078D078D078D07DE06E706F4068D07CB
:1006800001070A0717078D078D078D0724072D0718
:100690003A078D07470750075D078D078D078D07C0
:1006A0006A077307800781E090E0A0E0B0E08093E4
:1006B000490990934A09A0934B09B0934C090895B6
:1006C00010924D0910924E0910924F091092500944
:1006D00008951092510910925209109253091092E4
:1006E0005409089581E090E0A0E0B0E080935509BE
:1006F00090935609A0935709B09358090895109202
:10070000590910925A0910925B0910925C090895D8
:1007100083E090E0A0E0B0E080935D0990935E09F3
:10072000A0935F09B0936009089588E790E0A0E086
:10073000B0E08093750990937609A0937709B09300
:100740007809089588E790E0A0E0B0E08093790907
:1007500090937A09A0937B09B0937C09089588E768
:1007600090E0A0E0B0E080937D0990937E09A09393
:100770007F09B09380090895109285091092860927
:100780001092870910928809089510928909109291
:100790008A0910928B0910928C09089581E090E0EB
:1007A000A0E0B0E080938D0990938E09A0938F090B
:1007B000B0939009089510929109109292091092A5
:1007C0009309109294090895109295091092960930
:1007D0001092970910929809089510929909109211
:1007E0009A0910929B0910929C09089510929D09F4
:1007F00010929E0910929F091092A00908951092DC
:10080000A1091092A2091092A3091092A4090895B7
:100810001092A5091092A6091092A7091092A80992
:1008200008951092AD091092AE091092AF0910927E
:10083000B00908951092B1091092B2091092B3094B
:100840001092B40908951092B5091092B609109249
:10085000B7091092B80908951092C5091092C609F7
:100860001092C7091092C80908951092C9091092F0
:10087000CA091092CB091092CC0908951092CD09A3
:100880001092CE091092CF091092D009089581E0FC
:1008900090E0A0E0B0E08093D9099093DA09A093AA
:1008A000DB09B093DC09089581E090E0A0E0B0E0BE
:1008B0008093DD099093DE09A093DF09B093E009EE
:1008C00008958CE291E0A0E0B0E08093ED09909370
:1008D000EE09A093EF09B093F00908958CE291E03E
:1008E000A0E0B0E08093F1099093F209A093F3099E
:1008F000B093F40908958CE291E0A0E0B0E0809319
:10090000F5099093F609A093F709B093F8090895B3
:100910001092FD091092FE091092FF091092000A30
:1009200008951092010A1092020A1092030A10927E
:10093000040A08951092050A1092060A1092070AF6
:100940001092080A08951092150A1092160A109231
:10095000170A1092180A08951092190A10921A0A8A
:1009600010921B0A10921C0A089581E090E0A0E00A
:10097000B0E080931D0A90931E0AA0931F0AB093C3
:10098000200A089585E090E0A0E0B0E08093250A79
:100990009093260AA093270AB093280A089585E029
:1009A00090E0A0E0B0E08093290A90932A0AA093F7
:1009B0002B0AB0932C0A089589E190E0A0E0B0E002
:1009C00080932D0A90932E0AA0932F0AB093300A99
:1009D000089582E390E0A0E0B0E080933D0A909318
:1009E0003E0AA0933F0AB093400A089582E390E044
:1009F000A0E0B0E08093410A9093420AA093430A9A
:100A0000B093440A089582E390E0A0E0B0E08093C0
:100A1000450A9093460AA093470AB093480A08955E
:100A200082E390E0A0E0B0E080934D0A90934E0AFC
:100A3000A0934F0AB093500A089582E390E0A0E09B
:100A4000B0E08093510A9093520AA093530AB09356
:100A5000540A089582E390E0A0E0B0E08093550A44
:100A60009093560AA093570AB093580A089580E9C4
:100A700091E0A0E0B0E08093650A9093660AA093AD
:100A8000670AB093680A089580E991E0A0E0B0E0B9
:100A90008093690A90936A0AA0936B0AB0936C0AD8
:100AA000089580E991E0A0E0B0E080936D0A909312
:100AB0006E0AA0936F0AB093700A08951092750A97
:100AC0001092760A1092770A1092780A089510927E
:100AD000790A10927A0A10927B0A10927C0A089581
:100AE00010927D0A10927E0A10927F0A1092800A5C
:100AF000089510928D0B10928E0B10928F0B109206
:100B0000900B08951092910B1092920B1092930BF0
:100B10001092940B08951092950B1092960B1092D0
:100B2000970B1092980B089588E592E0A0E0B0E052
:100B300080938D0A90938E0AA0938F0AB093900AA7
:100B4000089588E592E0A0E0B0E08093910A909348
:100B5000920AA093930AB093940A089588E592E0CC
:100B6000A0E0B0E08093950A9093960AA093970A2C
:100B7000B093980A08958EE190E0A0E0B0E08093F1
:100B80009D0A90939E0AA0939F0AB093A00A08958D
:100B90008EE190E0A0E0B0E08093A10A9093A20AD9
:100BA000A093A30AB093A40A08958EE190E0A0E078
:100BB000B0E08093A50A9093A60AA093A70AB093E9
:100BC000A80A08951092B50A1092B60A1092B70AB0
:100BD0001092B80A08951092B90A1092BA0A1092A7
:100BE000BB0A1092BC0A08951092BD0A1092BE0A68
:100BF0001092BF0A1092C00A08951092DD0A109256
:100C0000DE0A1092DF0A1092E00A08951092E10ABB
:100C10001092E20A1092E30A1092E40A08951092E8
:100C2000E50A1092E60A1092E70A1092E80A08957F
:100C30001092ED0A1092EE0A1092EF0A1092F00A4A
:100C400008951092F10A1092F20A1092F30A10928B
:100C5000F40A08951092F50A1092F60A1092F70A13
:100C60001092F80A089585E090E0A0E0B0E080934B
:100C7000050B9093060BA093070BB093080B0895F8
:100C800085E090E0A0E0B0E08093090B90930A0B20
:100C9000A0930B0BB0930C0B089585E090E0A0E0BF
:100CA000B0E080930D0B90930E0BA0930F0BB093BD
:100CB000100B089584EB95E1A0E0B0E08093150B54
:100CC0009093160BA093170BB093180B089584EB19
:100CD00095E1A0E0B0E08093190B90931A0BA093DC
:100CE0001B0BB0931C0B089584EB95E1A0E0B0E0E2
:100CF00080931D0B90931E0BA0931F0BB093200BA2
:100D0000089585E090E0A0E0B0E080932D0B9093F3
:100D10002E0BA0932F0BB093300B089585E090E03D
:100D2000A0E0B0E08093310B9093320BA093330B93
:100D3000B093340B089585E090E0A0E0B0E080939C
:100D4000350B9093360BA093370BB093380B089567
:100D500010923D0B10923E0B10923F0B1092400BE5
:100D600008951092410B1092420B1092430B109277
:100D7000440B08951092450B1092460B1092470BAE
:100D80001092480B08951092550B1092560B10922A
:100D9000570B1092580B08951092590B10925A0B42
:100DA00010925B0B10925C0B089510925D0B1092E9
:100DB0005E0B10925F0B1092600B089510926D0CF9
:100DC00010926E0C10926F0C1092700C08958CE3C0
:100DD00090E0A0E0B0E08093710C9093720CA0932F
:100DE000730CB093740C089581E090E0A0E0B0E043
:100DF0008093750C9093760CA093770CB093780C3D
:100E0000089510927D0C10927E0C10927F0C10921F
:100E1000800C08958CE390E0A0E0B0E08093810C1A
:100E20009093820CA093830CB093840C089581E07E
:100E300090E0A0E0B0E08093850C9093860CA093A6
:100E4000870CB093880C08951092950C1092960C14
:100E50001092970C1092980C08958CE390E0A0E00B
:100E6000B0E08093990C90939A0CA0939B0CB09354
:100E70009C0C089581E090E0A0E0B0E080939D0C90
:100E800090939E0CA0939F0CB093A00C0895109289
:100E9000A50C1092A60C1092A70C1092A80C089505
:100EA0008CE390E0A0E0B0E08093A90C9093AA0CB2
:100EB000A093AB0CB093AC0C089581E090E0A0E05F
:100EC000B0E08093AD0C9093AE0CA093AF0CB093B8
:100ED000B00C08951092BD0C1092BE0C1092BF0C75
:100EE0001092C00C08958CE390E0A0E0B0E08093F5
:100EF000C10C9093C20CA093C30CB093C40C089582
:100F000081E090E0A0E0B0E08093C50C9093C60C27
:100F1000A093C70CB093C80C0895220F331F220F63
:100F2000331FF901E75BF64F1082118212821382A0
:100F30000895AF92BF92CF92DF92EF92FF920F93FC
:100F40001F93CF93DF936C017B018B01040F151F5F
:100F5000EB015E01AE18BF08C017D10759F06991C7
:100F6000D601ED91FC910190F081E02DC60119951B
:100F7000892B79F7C501DF91CF911F910F91FF90D8
:100F8000EF90DF90CF90BF90AF900895FC01538D0C
:100F9000448D252F30E0842F90E0821B930B541753
:100FA00010F0CF96089501970895FC01918D828DE0
:100FB000981761F0A28DAE0FBF2FB11D5D968C9179
:100FC000928D9F5F9F73928F90E008958FEF9FEFB8
:100FD0000895FC01918D828D981731F0828DE80F74
:100FE000F11D858D90E008958FEF9FEF0895FC012E
:100FF000918D228D892F90E0805C9F4F821B9109FB
:101000008F739927089581ED9CE0F1DF21E0892B12
:1010100009F420E0822F0895FC01A48DA80FB92FB8
:10102000B11DA35ABF4F2C91848D90E001968F7310
:101030009927848FA689B7892C93A089B1898C912F
:10104000837080648C93938D848D981306C002887E
:10105000F389E02D80818F7D80830895EF92FF9248
:101060000F931F93CF93DF93EC0181E0888F9B8DCB
:101070008C8D98131AC0E889F989808185FF15C085
:101080009FB7F894EE89FF896083E889F9898081A8
:101090008370806480839FBF81E090E0DF91CF9177
:1010A0001F910F91FF90EF900895F62E0B8D10E099
:1010B0000F5F1F4F0F731127E02E8C8D8E110BC009
:1010C0000FB607FCFACFE889F989808185FFF5CF53
:1010D000CE01A2DFF2CFEB8DEC0FFD2FF11DE35A15
:1010E000FF4FF0829FB7F8940B8FEA89FB898081CC
:1010F0008062D0CF682F81ED9CE0B0CFCF93DF939B
:10110000EC01888D8823B1F0AA89BB89E889F98927
:101110008C9185FD03C0808186FD0CC00FB607FC55
:10112000F7CF8C9185FFF2CF808185FFEDCFCE0187
:1011300073DFEACFDF91CF91089580E090E0892BB3
:1011400021F061DF81110E94000080E090E0892B96
:1011500049F080E090E0892B29F00E940000811185
:101160000E94000080E090E0892B49F080E090E050
:10117000892B29F00E94000081110E94000080E06C
:1011800090E0892B49F080E090E0892B29F00E94C3
:10119000000081110C94000008958150823108F004
:1011A0005AC0E82FF0E08827E752F74F8F4F0C9492
:1011B0006357F908FD08EB08F108F5082B09000949
:1011C00006090A091009140918091E0922092B0920
:1011D00026092C093009809180008F778093800048
:1011E0000895809180008F7DF9CF80918000877F66
:1011F000F5CF84B58F7784BD089584B58F7DFBCFFF
:101200008091B0008F778093B00008958091B000F6
:101210008F7DF9CF809190008F7780939000089513
:10122000809190008F7DF9CF80919000877FF5CFDE
:101230008091A0008F778093A00008958091A000F6
:101240008F7DF9CF8091A000877FF5CF809120011D
:101250008F77809320010895809120018F7DF9CFB1
:1012600080912001877FF5CFCF93DF93282F30E047
:10127000F901E35BFD4F8491F901E355FD4FD491F2
:10128000F901ED50FD4FC491CC2399F0811185DF18
:10129000EC2FF0E0EE0FFF1FED5CFD4FA591B49138
:1012A000EC91ED2381E090E009F480E0DF91CF91B3
:1012B000089580E090E0FACF1F93CF93DF93282F1B
:1012C00030E0F901E35BFD4F8491F901E355FD4FF7
:1012D000D491F901ED50FD4FC491CC23A1F0162F0C
:1012E00081115BDFEC2FF0E0EE0FFF1FE75EFD4F9B
:1012F000A591B4918FB7F894EC91111108C0D095D5
:10130000DE23DC938FBFDF91CF911F910895DE2BF9
:10131000F8CFCF93DF9390E0FC01E355FD4F24918C
:101320008D509D4FFC0184918823C9F090E0880F77
:10133000991FFC01ED56FD4FA591B491FC01E75EAC
:10134000FD4FC591D49161110DC09FB7F8948C9158
:10135000209582238C938881282328839FBFDF9147
:10136000CF910895623051F49FB7F8943C91822F49
:10137000809583238C93E8812E2BEFCF8FB7F89441
:10138000EC912E2B2C938FBFEACFCF938CB58C6032
:101390008CBD8CB58F7D8CBD8CB58C7F8CBD8DB597
:1013A0008E7F8DBDCFB7F89480914209811123C003
:1013B000E8E2F3E08491E2EEF2E09491E82FF0E0CD
:1013C000EE0FFF1FED56FD4FA591B491EC91E9236F
:1013D00019F461E085E370DF61E085E39ADF8CB5A5
:1013E00080618CBD8CB580648CBD61E084E391DF4D
:1013F00061E083E38EDF809142098F5F8093420931
:10140000CFBFCF9108958230910538F0880F991F92
:10141000880F991F05970197F1F708953FB7F89442
:101420008091280890912908A0912A08B0912B0852
:1014300026B5A89B05C02F3F19F00196A11DB11D2F
:101440003FBFBA2FA92F982F8827BC01CD01620F6B
:10145000711D811D911D42E0660F771F881F991F26
:101460004A95D1F708958F929F92AF92BF92CF92F3
:10147000DF92EF92FF926B017C01D0DF4B015C01A8
:10148000C114D104E104F104B1F0C8DF681979098D
:101490008A099B09683E73408105910588F321E024
:1014A000C21AD108E108F10888EE880E83E0981E80
:1014B000A11CB11CE5CFFF90EF90DF90CF90BF90C3
:1014C000AF909F908F9008952FB7F8946091240863
:1014D0007091250880912608909127082FBF0895C4
:1014E000CF92DF92EF92FF92CF93DF93EC016032C5
:1014F00082E07807CCF5653B710514F064EB70E091
:10150000898128E830E0281B310987FD3395220FB7
:10151000331F220F331F6901330FEE08FF088A8142
:1015200028E532E0281B310987FD3395220F331F50
:10153000220F331F032E000C440B550B2C193D09B1
:101540004E095F09DB0177FF02C0B0E0A0E00E9416
:101550000B5624EB30E040E050E00E94E555C20E0F
:10156000D31EE41EF51EB601E881E03370F5298133
:1015700088E890E0821B910927FD9395880F991FB9
:10158000880F991F681779077CF02A8188E592E017
:10159000821B910927FD9395880F991F880F991F2A
:1015A000681779070CF4CB010297880F991F4FB782
:1015B000F8942E2F30E0F901EE0FFF1FE20FF31F1A
:1015C000E259F24F928381834FBFDF91CF91FF9019
:1015D000EF90DF90CF9008951F93CF93DF93EC01AE
:1015E000162F8881803308F04DC061E0812F91DE95
:1015F0008881282F30E0F901EE0FFF1FE20FF31F63
:10160000E259F24F1F736081607C612B6083198205
:101610001A822CE0622F0E945757829FB00111243A
:1016200030E020E0AB01420F531FFA01EE0FFF1F25
:10163000E40FF51FE259F24F908196FD16C02F5F1F
:101640003F4F2C30310571F7813009F51092800041
:1016500082E0809381001092850010928400B19AFC
:1016600080916F00826080936F00E8818E2F90E000
:10167000FC01EE0FFF1FE80FF91FE259F24F8081C6
:10168000806480838881DF91CF911F91089582309B
:1016900061F4109290008093910010929500109246
:1016A000940088BB80937100E0CF833069F410927E
:1016B000A00082E08093A1001092A5001092A400E7
:1016C00089BB80937200D1CF8111CFCF10922001BE
:1016D00082E08093210110922501109224018ABB9F
:1016E00080937300C2CFAF92BF92CF92DF92EF92FE
:1016F000FF920F931F93CF93DF936B017A01EC015D
:10170000C15ED74F28813CE0389F8001399F100D82
:101710001124A090FE0DB12C27FF1FC0FB011182E8
:10172000108288818F5F888388819801280F311DFE
:1017300087FD3A95F6012A153B051CF488818C300B
:10174000BCF180819181049680349C4908F471C079
:10175000F6018081918104966EC088819801280FDE
:10176000311D87FD3A952A153B05DCF68881A801D5
:10177000480F511D87FD5A95FA01EE0FFF1FE40F28
:10178000F51FE259F24F808186FFCBCF8881F801A7
:10179000E80FF11D87FDFA95CF01EE0FFF1FE80F4F
:1017A000F91FE259F24F808160E08F7385DDB9CF78
:1017B000808191812881A801420F511D27FD5A95F2
:1017C0009A01FA01EE0FFF1FE20FF31FE259F24FE9
:1017D00021813281820F931FF70191838083888159
:1017E0009801280F311D87FD3A95F901EE0FFF1F73
:1017F000E20FF31FE259F24F808186FF21C08881FA
:10180000080F111D87FD1A95F801EE0FFF1FE00F5D
:10181000F11FE259F24F808161E08F73DF91CF9128
:101820001F910F91FF90EF90DF90CF90BF90AF90FE
:1018300043CD80E49CE9F701918380838FEF888317
:10184000DF91CF911F910F91FF90EF90DF90CF909C
:10185000BF90AF900895089508950895089508954C
:10186000EBE0F1E08081877F80830895EBE0F1E099
:1018700080818860808308958E9808958E9A089557
:1018800014980895149A089588980895889A089548
:1018900060E0FC01818910CD60E0FC0183850CCD06
:1018A00061E0FC01818908CD61E0FC01838504CD04
:1018B000CF93DF93EC01FC01ED58FF4F1082379777
:1018C00081E0808360E08B85F7DC8D899E89892BA0
:1018D00029F060E08989DF91CF91EECCDF91CF9143
:1018E0000895CF93DF93EC01898DBEDC2C8D2817F2
:1018F000190621F48D8DDF91CF91089580E0FBCF03
:10190000CF93DF93EC018F89AFDC2C8D281719065C
:1019100021F48D8DDF91CF91089580E0FBCFCF939F
:10192000DF93EC018D859BA961E0911101C060E01E
:10193000C3DC8B899CA9992321F09DA961E09111B9
:1019400001C060E0DF91CF91B7CCCF93DF93EC0182
:101950008D859BA960E0911101C061E0ADDC8B89B0
:101960009CA9992321F09DA960E0911101C061E03B
:10197000DF91CF91A1CCCF93DF93EC0161E08F8514
:101980009BDC8CA9882319F061E08D8995DCCF5808
:10199000DF4F1882DF91CF910895CF93DF93EC0151
:1019A00060E08F8589DC8CA9882319F060E08D893F
:1019B00083DCCF58DF4F81E08883DF91CF9108959A
:1019C000CF92DF92EF92FF920F931F93CF93DF930B
:1019D000FC01DC01A05CBF4F4D935D936D937C9344
:1019E000139714964D935D936D937C931397149670
:1019F0000D931D932D933C931397EC01C45BDF4F24
:101A0000E88282AD882351F092A991114CC037FF32
:101A100050C01D921D921D921C92139743AD54AD60
:101A200065AD76AD14161506160617063CF597AD8E
:101A3000992321F10D911D912D913C9113976801EE
:101A4000790137FF07C0CC24DD247601C01AD10A02
:101A5000E20AF30A4C155D056E057F057CF437FF3D
:101A600007C070956095509541955F4F6F4F7F4FC0
:101A70004D935D936D937C931397892FDF01A75A44
:101A8000BF4F1D921D921D921C921397E759FF4F55
:101A900091E09083DF91CF911F910F91FF90EF9094
:101AA000DF90CF90089510161106120613060CF45D
:101AB000B0CF80E0B3CF0F931F93CF93DF93EC01B0
:101AC000062F8B8D81110DC0CE011ADF182FCE018C
:101AD00008DF0111182F812FDF91CF911F910F91F6
:101AE0000895CE01FEDE182FCE010ADFF2CFCF938C
:101AF000DF93EC01FC01ED58FF4F81E08083AE01E4
:101B00004C5B5F4FFA0180819181A281B3819E017C
:101B100026593F4FF9012081222309F440C0019644
:101B2000A11DB11DFA0180839183A283B383FE01BD
:101B3000EA58FF4F20813181C901959587958C0F17
:101B40009D1F32970190F081E02D20FF08C0DC013D
:101B50002D913C91E20FF31F0190F081E02D19953A
:101B60008D899E89892BF9F0FE01E658FF4F20816F
:101B70003181C901959587958C0F9D1FC858DF4FFE
:101B8000E881F98120FF08C0DC012D913C91E20F32
:101B9000F31F0190F081E02DDF91CF91199401970F
:101BA000A109B109BFCFDF91CF9108958F929F9284
:101BB000AF92BF92CF92DF92EF92FF920F931F935B
:101BC000CF93DF93EC01FC01E75AFF4F60817181F5
:101BD000828193810E94B7546B017C016EA97FA919
:101BE00088AD99AD0E94B9549B01AC0160E074E2EC
:101BF00084E799E40E94A7564B015C01FE01EB5972
:101C0000FF4F60817181828193810E94B7549B0153
:101C1000AC01C501B4010E94A7564B015C018E01C5
:101C2000035A1F4F20E030E040E05FE30E94185568
:101C3000A70196010E9443560E941457F801608341
:101C4000718382839383CF59DF4FA5019401C7012C
:101C5000B6010E9443560E941457688379838A8391
:101C60009B83DF91CF911F910F91FF90EF90DF90B9
:101C7000CF90BF90AF909F908F9008950F931F9338
:101C8000CF93DF93FC01ED58FF4F20812223B9F061
:101C90007A97008111812281338138964081518168
:101CA00062817381041715072607370710F1EC01CD
:101CB000FFDDCE01DF91CF911F910F9177CFFC0116
:101CC000E759FF4F20812223A1F0709700811181F5
:101CD000228133813496408151816281738104175E
:101CE00015072607370728F0DF91CF911F910F9135
:101CF000FECEDF91CF911F910F910895FC01E7591E
:101D0000FF4F2081222361F0709780819181A28111
:101D1000B3810196A11DB11D80839183A283B383FA
:101D200008950F931F93FC01E45BFF4F2081211165
:101D300012C038970081118122813381349640810D
:101D400051816281738104171507260737073CF418
:101D50001F910F91FACDFC0122A92111F9CF1F91FA
:101D60000F91DDCDFC0181E086838783118610868B
:101D700012868CE291E0A0E0B0E0868F978FA0A35E
:101D8000B1A342E350E060E070E042A353A364A338
:101D900075A346A357A360A771A782A793A7A4A77B
:101DA000B5A788E790E0A0E0B0E086A797A7A0AB32
:101DB000B1AB12AA13AA14AA15AA84E690E0A0E077
:101DC000B0E086AB97ABA0AFB1AF12AE13AE14AE1E
:101DD00015AE16AE17AEDF01A05CBF4F1D921D926F
:101DE0001D921C92139714961D921D921D921C9287
:101DF000139714961D921D921D921C921397149680
:101E00001C9211961D921D921D921C92139714966E
:101E10001D921D921D921C92139714961D921D9255
:101E20001D921C92139714961D921D921D921C9246
:101E3000139714961D921D921D921C92139714963F
:101E40001D921D921D921C92139714961D921D9225
:101E50001D921C92139714961C9211961C92119627
:101E60001C9211961C9211961C9211961C9211961E
:101E70001C9211961C9211961C9211961C9211960E
:101E80001C921486138616861586108A1786128A67
:101E9000118A148A138A168A158A108E178A128E4E
:101EA000118E119684E59CE011969C938E93129668
:101EB00011961C921E92129680E59CE011969C93BE
:101EC0008E93129611961C921E9212968CE49CE0B0
:101ED00011969C938E93129611961C921E921296B6
:101EE00088E49CE08D939C93EE57FF4F1182108203
:101EF00008950895089508958FEF9FEF0895089528
:101F000008954F925F926F927F928F929F92AF92BD
:101F1000BF92CF92DF92EF92FF92CF93DF93EC01CB
:101F20006C897D898E899F8988889988AA88BB88D1
:101F3000CE8CDF8C0D2C000CEE08FF08603127E200
:101F400072078105910529F016161706180619065D
:101F5000ACF0A7019601C501B4010E944857DF917A
:101F6000CF91FF90EF90DF90CF90BF90AF909F9078
:101F70008F907F906F905F904F9008950E94B9541A
:101F800020E030E44CE156E40E94A7562B013C01CE
:101F9000488E598E6A8E7B8EC501B4010E94B95459
:101FA000A30192010E9418554B015C01C701B601C3
:101FB0000E94B9549B01AC01C501B4010E9418559F
:101FC0000E940F57CCCFFC01118210821382128223
:101FD0001582148217821682108611861286138645
:101FE0001486158616861786108A118A128A138A15
:101FF000108E118E128E138E158E148E178E168ED5
:1020000010A211A212A213A214A215A216A217A224
:1020100010A611A612A613A614A615A681E090E09C
:1020200097A786A780E197E2A0E0B0E0848B958B2C
:10203000A68BB78B08958EBD00000DB407FEFDCFB3
:102040008EB50895DF92EF92FF920F931F93CF9377
:10205000DF93EC01D62E122F032FF42EE52E60E035
:1020600088852AD98D2D8068E6DF89878E2DE3DF6C
:102070008F2DE1DF802FDFDF812FDDDF61E08885BD
:102080001BD98985DF91CF911F910F91FF90EF9020
:10209000DF9008953F924F925F926F927F928F925E
:1020A0009F92AF92BF92CF92DF92EF92FF920F93E7
:1020B0001F93CF93DF9300D000D0CDB7DEB79E83C0
:1020C0008D83362E49015A01270138015ED960E01F
:1020D000ED81FE818085F0D8832DADDFED81FE811D
:1020E000818780E0A8DF80E0A6DF80E0A4DF80E0D9
:1020F000A2DF61E0ED81FE818085DED860E0ED81C8
:10210000FE818085D9D8832D96DFED81FE81818780
:1021100080E091DFF82E80E08EDF082F80E08BDFFB
:10212000182F80E088DF202F30E050E040E03F298A
:1021300069017A01FE2CED2CDC2CCC24C12AFE2C6A
:10214000ED2CDC2CCC24C82A61E0ED81FE81808559
:10215000B3D88C249D24AE24BF24482059206A2063
:102160007B20A30192012C253D254E255F25632D63
:102170008D819E8167DFED81FE81818526960FB678
:10218000F894DEBF0FBECDBFDF91CF911F910F91AD
:10219000FF90EF90DF90CF90BF90AF909F908F9087
:1021A0007F906F905F904F903F900895CF93DF9313
:1021B000EC0160E0888580D880E03DDF898780E0A1
:1021C0003ADF80E038DF80E036DF80E034DF61E056
:1021D000888572D88985DF91CF9108958F929F92DB
:1021E000AF92BF92CF92DF92EF92FF920F931F9325
:1021F000CF93DF93F7016081662389F169017A014A
:10220000EC0188819981D2DF482F50E0CA01959571
:10221000879595958795CC5BDF4F80FD07C083E060
:10222000559547958A95E1F740FF26C020E030E0BC
:1022300040E85FE3F70160817181828193810E94B0
:102240004356F7016083718382839383F601808113
:102250009181A281B38188839983AA83BB83DF9113
:10226000CF911F910F91FF90EF90DF90CF90BF9093
:10227000AF909F908F900895F70180809180A28009
:10228000B38020E030E0A901C501B4010E944057AD
:10229000181674F4F8012081318142815381C501FF
:1022A000B4010E944256F701608371838283938355
:1022B00088819981AA81BB81F60180839183A28361
:1022C000B383CDCFCF93DF93EC0161E0888521D834
:1022D00061E088850E945C0958D8CE01DF91CF91DA
:1022E00065CFCF93DF93EC018C818835A9F58DEC18
:1022F00092E1998388838DEF92E19B838A8384E5C1
:102300009CE0FE01EC58FF4F91838083329611824E
:10231000108280E59CE03296918380833296118210
:1023200010828CE49CE032969183808332961182F5
:10233000108288E49CE032969183808332961182E9
:10234000108288819981BEDF8C81883589F48A81E9
:102350009B81DF91CF91B6CF893529F48DED92E144
:1023600099838883CCCF8A3551F68DEE92E1F8CFF0
:10237000DF91CF9108958F929F92AF92BF92CF92AB
:10238000DF92EF92FF920F931F93CF93DF93EC01B5
:102390008B015A01690196DF85E090E0A0E0B0E092
:1023A00008301105C1F1B4F487E090E0A0E0B0E09E
:1023B0000230110581F186E090E0A0E0B0E0043049
:1023C000110549F101301105A1F488E090E0A0E089
:1023D000B0E021C083E090E0A0E0B0E00032110561
:1023E000D1F05CF484E090E0A0E0B0E000311105B1
:1023F00091F080E090E0DC010EC082E090E0A0E08F
:10240000B0E00034110539F081E090E0A0E0B0E0E8
:102410000038110571F7582F442733272227E12C64
:10242000F12C00E01FE06CE6CE0134DEB50190E057
:1024300080E00E94B75425ED34E045E352E40E9469
:10244000185520E030E04AE754E40E94A75628EBF4
:102450003EE145E05EE30E9418554B015C0126E633
:1024600036E646EA5EE30E94A75620E030E040E808
:102470005FE30E9442560E941457603180F42CEEB4
:1024800031E548E35EE3C501B4010E94A75620E0B0
:1024900030E040E85FE30E9442560E941457862FC6
:1024A0008F71262F30E050E040E0542F432F322F21
:1024B000222722273F7144275527282B60E1CE0190
:1024C000C1DD0D2C000CEE08FF08A60133272227E2
:1024D000E12CF12C01E010E06CE6CE01DBDDE12C1B
:1024E000F12C8701E39421E030E040E050E060E02F
:1024F000CE01D0DD1FE0E12EF12C00E010E023E062
:1025000030E040E050E06CE6CE01C4DDE12C10E8A4
:10251000F12E01E010E020E030E840E050E06CE611
:10252000CE01B8DDE12CF12C8701F39420E031E0FD
:1025300040E050E060E0CE01ADDDE12C14E0F12E92
:1025400000E010E020E034E040E050E060E0CE0148
:10255000A1DD2FEF3FEF4FE050E064E1CE0172DDEF
:1025600020E030E0A90165E1CE016CDD1FE0E12E45
:10257000F12C00E010E025E030E040E050E06CE6B7
:10258000CE0188DDE12CF12C8701F39420E032E0CC
:1025900040E050E06CE6CE017DDDE12C10E2F12E52
:1025A00000E010E020E030E240E050E06CE6CE01D8
:1025B00071DD64E670E080E090E0DF91CF911F91E3
:1025C0000F91FF90EF90DF90CF90BF90AF909F90D2
:1025D0008F900C94330ACF92DF92EF92FF920F9379
:1025E0001F93CF93DF93EC017B016A0189019A016C
:1025F000AB01B80188819981BEDE8C81883571F488
:102600009601A701B8018A819B81DF91CF911F912B
:102610000F91FF90EF90DF90CF90ADCEDF91CF91F3
:102620001F910F91FF90EF90DF90CF900895089544
:1026300008950895089508950F931F93CF93DF93FE
:102640008B01EA01AB01415051094433510508F0B7
:10265000ECC02230310508F0E8C048E3429FF001A9
:10266000439FF00D1124E80FF91FE60FF71F81E0DB
:1026700080836C2F232B09F4D4C061E0802F0E944B
:102680008909209751F460E0802F0E945C09CE01F7
:10269000DF91CF911F910F910895CF3FD10511F494
:1026A00061E0BFC0F801E35BFD4FE491E150E2312E
:1026B00008F0B2C0F0E08827EF59FC4E8F4F0C9421
:1026C000635773137A137F13891393130C149D1399
:1026D000A513AD13B713C113CB13DA13E4130C1402
:1026E000EE13F813021484B5806884BDC7BDD0E032
:1026F000C0E0CDCF84B5806284BDC8BDF8CF8091E5
:102700008000806880938000D0938900C093880007
:10271000EECF80918000806280938000D0938B0008
:10272000C0938A00E4CF809180008860809380000D
:10273000D0938D00C0938C00DACF8091B000806878
:102740008093B000C093B300D2CF8091B00080627C
:102750008093B000C093B400CACF8091900080688D
:1027600080939000D0939900C0939800C0CF80913F
:102770009000806280939000D0939B00C0939A0059
:10278000B6CF80919000886080939000D0939D0098
:10279000C0939C00ACCF8091A00080688093A00083
:1027A0008091A0008F7B8093A000D093A900C0935C
:1027B000A8009DCF8091A00080628093A000D0935C
:1027C000AB00C093AA0093CF8091A0008860809353
:1027D000A000D093AD00C093AC0089CF80912001C0
:1027E000806880932001D0932901C09328017FCF76
:1027F00080912001806280932001D0932B01C093AF
:102800002A0175CF80912001886080932001D093A8
:102810002D01C0932C016BCF60E0C038D1050CF0C6
:102820003FCF802F0E945C0962CFC1E0D0E02FCF64
:102830000895CF93DF93D0E0C0E0CE010E94D10194
:10284000882319F0CE010E9467022196C13ED1056E
:10285000A1F7DF91CF9108950895CF93DF93EC0115
:10286000FC01EE5DFC4F1082EE58F1098081811170
:1028700003C0CE0140967FD8FE01EB56FD4F80810C
:10288000811104C0CE018C569F4F75D8FE01EA56C7
:10289000FD4F8081811104C0CE01885E9E4F6BD8B0
:1028A00064E670E080E090E0DF91CF910C94330A11
:1028B0000895089508950895089580911D089091B0
:1028C0001E08892B09F040C08FE090E00E943A4F2B
:1028D000FC0181E090E0A0E0B0E080839183A283DE
:1028E000B38384839583A683B78380879187A287E8
:1028F000B38715861486168610922E0910922F091A
:102900001092300910923109109232091092330955
:102910001092340910923509109236091092370935
:1029200010923809109239091092CD0C1092CE0CE9
:102930001092CF0C1092D00C10925E0810925D088D
:10294000F0931E08E0931D0880911D0890911E08C9
:102950000895B3DF85E40E94340921E0892B09F44E
:1029600020E020934309A9DF84E40E94340921E098
:10297000892B09F420E0209344099FDF83E40E941F
:10298000340921E0892B09F420E02093450995DFE3
:1029900082E40E94340921E0892B09F420E020938D
:1029A00046098BDF81E40E94340921E0892B09F478
:1029B00020E02093470981DF80E40E94340921E070
:1029C000892B09F420E020934809089576DFC1CFD0
:1029D00074DFFC01168690E080E00895809119086C
:1029E00090911A08892B41F481E090E00E943A4FBF
:1029F00090931A08809319088091190890911A08E9
:102A000008950F931F93CF93DF938B01E7DFF801B6
:102A1000C2A1D3A1868D978D8530910529F14CF403
:102A20000497B1F090E080E0DF91CF911F910F917A
:102A300008958630910511F10B97A1F767E070E0DA
:102A400088E09EE00E94EC0ABE0188E09EE009C09A
:102A500064E070E08FEF9DE00E94EC0ABE018FEF12
:102A60009DE00E94700ADECF65E070E082E09EE0AB
:102A70000E94EC0ABE0182E09EE0F3CF66E070E0C7
:102A800085E09EE00E94EC0ABE0185E09EE0E9CF71
:102A90008091160890911708892B91F480E790E0B7
:102AA0000E943A4FFC0131969C012B5C3F4F1192E2
:102AB00017AAE217F307D9F790931708809316081F
:102AC00080911608909117080895CF93DF93EB013A
:102AD000DFDF6AA98E8D0E94890990E080E0DF9196
:102AE000CF9108954F925F926F927F92AF92BF9273
:102AF000CF92DF92EF92FF920F931F93CF93DF93CA
:102B0000EB01C6DF8C01CAA8DBA84EA45FA468A8AD
:102B100079A8AEA0BFA0EE8CFF8C4AA15BA1960164
:102B2000B7018ADDC301B2010E94330A9601A501F3
:102B3000B701C80181DD90E080E0DF91CF911F9166
:102B40000F91FF90EF90DF90CF90BF90AF907F906C
:102B50006F905F904F900895CF93DF93EB0198DFD4
:102B60002AA93BA94AA15BA16E8D7F8D65DD90E00E
:102B700080E0DF91CF910895FC0101900020E9F7FA
:102B80003197AF01481B590BBC0181ED9CE00C94BF
:102B900099078F929F92AF92BF920F931F93CF93FB
:102BA000DF93CDB7DEB7A1970FB6F894DEBF0FBEA7
:102BB000CDBF19A2423008F44AE08E010F5D1F4FCD
:102BC000842E912CB12CA12CA50194010E941156A8
:102BD000E62FB901CA01EA30ECF4E05DD801EE93CA
:102BE0008D01232B242B252B79F790E080E0109783
:102BF00011F0CD01C1DFA1960FB6F894DEBF0FBE74
:102C0000CDBFDF91CF911F910F91BF90AF909F905B
:102C10008F900895E95CE2CFCF92DF92EF92FF921E
:102C2000CF93DF9397FF18C06B017C018DE20E9468
:102C30007A08EC0166277727CB016C197D098E098C
:102C40009F094AE0A6DF8C0F9D1FDF91CF91FF9077
:102C5000EF90DF90CF9008954AE0DF91CF91FF9001
:102C6000EF90DF90CF9095CFBC01990F880B990B17
:102C7000D3CF82CF88E893E0FCDF6091CD0C7091D8
:102C8000CE0C8091CF0C9091D00CC6DF8EED97E0EA
:102C9000F0CF882319F08AE697E0EBCF83E697E040
:102CA000FCCF0F931F93CF93DF938C01EB018AE648
:102CB00093E0DFDF82E194E0DCDFF80184810E94B1
:102CC0007A08CE01D1DFF9DDDF91CF911F910F910D
:102CD000D1CFEF92FF920F931F93CF93DF93182FD3
:102CE000092F7B016115710569F50E94340931E0F6
:102CF00020E0019709F030E0C32FD22F82E0E816E0
:102D0000F10408F045C08BE893E0B3DF82E194E082
:102D1000B0DF8FE893E0ADDF812F902FA5DF82E158
:102D200094E0A7DF8FE098E0A4DFCE019DDFC5DD52
:102D3000A1DF90E080E0DF91CF911F910F91FF9094
:102D4000EF900895D0E0C0E061307105B9F6812FB1
:102D5000163310F08AEC810F20917B00982F987029
:102D6000277F922B90937B008770806480937C00F8
:102D700080917A00806480937A0080917A0086FD49
:102D8000FCCF80917800C0917900DC2FC82FB6CF9E
:102D900081E090E0D0CF0F931F93CF93DF93FC019E
:102DA0002081318121153105C1F1EC01822F0E9472
:102DB000340921E0892B09F420E02B876A85261746
:102DC00001F11E821F82188619860E811F812885B7
:102DD00039858A819B81AC81BD81081719072A0733
:102DE0003B07DCF081E0682788810E945C0950DEA7
:102DF00070E060E088819981DF91CF911F910F9100
:102E000068CF8E819F81A885B9850196A11DB11DCE
:102E10008E839F83A887B987D8CFDF91CF911F91E9
:102E20000F910895CF93DF93EB0132DE6AA97BA95E
:102E30008E8D9F8D4EDF90E080E0DF91CF910895E1
:102E40002F923F924F925F926F927F928F929F92BA
:102E5000AF92BF92CF92DF92EF92FF920F931F93A8
:102E6000CF93DF93CDB7DEB762970FB6F894DEBF8E
:102E70000FBECDBF1C018C010C5B1F4F1E870D8741
:102E8000D8014D915D916D917C917C01B8E4EB0E80
:102E9000F11CF70180819181A281B3816101FCE481
:102EA000CF0ED11CF60120810A5D1F4F58017F967D
:102EB0004F012223A1F1F10122A9F801208321E091
:102EC000F4012083411551056105710559F4F101A3
:102ED00002A113A124A135A1EB59FF4F0083118357
:102EE000228333838101005C1F4FF80140805180B1
:102EF00062807380910127593F4F59014816590646
:102F00006A067B06B4F5481759076A077B07DCF1A8
:102F1000D6018C91811137C0D5011C923CC121E0B2
:102F2000481759076A077B070CF020E0F50120835A
:102F30002A013B0177FF07C0442455243201441A7B
:102F4000550A660A770A8C019D01B7FF07C0002762
:102F500011279801081B190B2A0B3B0BBB24B394B8
:102F600040165106620673060CF4B12CF401B082CF
:102F7000A9CF84159505A605B70554F684179507BE
:102F8000A607B7072CF6F5018081882329F2D60120
:102F90008C9181110EC0F60180818111BDCFD401C9
:102FA0006C9181E06827C1010E945B0D8111B4CF53
:102FB00006C060E0C1010E945B0D8111ECCFD10120
:102FC0009A962D913D914D915C919D9729833A83DD
:102FD0004B835C835E962D913D914D915C919197D1
:102FE0002D833E834F83588792962D913D914D912D
:102FF0005C91959729873A874B875C87F701808199
:103000009181A281B381ED85FE85C080D180E2806F
:10301000F380F8014081518162817381F101E359AC
:10302000FF4F1082319610823101FFE66F0E711C46
:10303000F3011082910120593F4FF901108232961D
:1030400010824C015D01841A950AA60AB70AB7FEE0
:1030500008C0B094A09490948094811C911CA11CF1
:10306000B11C481759076A077B072CF0C81AD90A00
:10307000EA0AFB0A04C0C41AD50AE60AF70AD5010F
:10308000C401B595A795979587958D879E87AF873E
:10309000B88B81010E581F4F8C149D04AE04BF04E1
:1030A00008F09FC0D10196960D90BC91A02DBA8BCF
:1030B000A98B81E0F9018083D8018C93F10182858D
:1030C000882309F45CC00E94640AD10118960D910E
:1030D0001C91012E000C220B330B601B710B820B19
:1030E000930B693E73408105910508F448C00E9426
:1030F000640AF1017187608781E993E0BADD85E9AF
:1031000093E0B7DD60E070E0CB0186DD8BE993E012
:10311000B0DDC701B60180DD81EA93E0AADDC5011B
:10312000B4017ADD87EA93E0A4DD4AE06D857E850F
:103130008F8598892EDD8EEA93E09BDD69817A8107
:103140008B819C8169DD84EB93E093DD69857A85D1
:103150008B859C8561DD8AEB93E08BDD6D817E81C3
:103160008F81988559DD80EC93E083DD82E194E0E6
:1031700080DD89899A8978DD8EED97E07ADDF1012D
:10318000EB59FF4F09891A89C801B0E0A0E080839C
:103190009183A283B38360E0C1010E945B0D882309
:1031A00039F0F101EC5BFF4F108211821282138221
:1031B00062960FB6F894DEBF0FBECDBFDF91CF9100
:1031C0001F910F91FF90EF90DF90CF90BF90AF9045
:1031D0009F908F907F906F905F904F903F902F9037
:1031E00008952D853E854F8558892C153D054E0542
:1031F0005F0508F450C089819A81AB81BC818C1530
:103200009D05AE05BF0544F4AD81BE811196BA8B14
:10321000A98B81E0F3014FCFC701B6010E94B954D9
:103220002B013C0169817A818B819C810E94B95478
:103230009B01AC01C301B2010E94A7562B013C01C6
:103240006D817E818F81988529853A854B855C8546
:10325000621B730B840B950B0E94B9549B01AC014C
:10326000C301B2010E9418552B013C0169857A8582
:103270008B859C850E94B9549B01AC01C301B201AE
:103280000E9443560E940F577A8B698B81E0F101AF
:10329000E359FF4F10CFD501C40129813A814B81F9
:1032A0005C81821B930BA40BB50BC816D906EA06EA
:1032B000FB065CF44D815E814E5F5F4F5A8B498BFC
:1032C00081E0F101E159FF4FF6CEC501B4016C195F
:1032D0007D098E099F090E94B9542B013C01698127
:1032E0007A818B819C810E94B9549B01AC01C301FE
:1032F000B2010E94A7562B013C016D817E818F8116
:10330000988529853A854B855C85621B730B840BF8
:10331000950B0E94B9549B01AC01C301B2010E94FC
:1033200018552B013C0169857A858B859C850E9407
:10333000B9549B01AC01C301B2010E9443560E94E3
:103340000F577A8B698B81E0F101E259FF4FB3CEC1
:10335000CF93DF9386EC93E08CDC8AEC93E089DCFE
:10336000C3E4D9E0888195DC8EEC93E082DC89812E
:1033700090DC82ED93E07DDC8A818BDC86ED93E04E
:1033800078DC8B8186DC8AED93E073DC8C8181DCD8
:103390008EED93E06EDC8D817CDCDF91CF916ACC89
:1033A0008CDAD6CF82EE93E064DC87DAD2DA85DA83
:1033B000CFDF6EDB70E060E088E090E08ADC68DB05
:1033C00070E060E089E090E084DC62DB70E060E067
:1033D0008AE090E07EDC5CDB70E060E08DE090E015
:1033E00078DC90E080E00895CF92DF92EF92FF9238
:1033F000CF93DF93EB01CB010E94D101882351F1E0
:10340000FE01EE0FFF1FEE0FFF1FE75BF64FC080C0
:10341000D180E280F38089EE93E02BDC82E194E0BE
:1034200028DC8FE893E025DCCE011EDC82E194E00D
:1034300020DC8FE098E01DDCC701B601EDDB3DDA52
:1034400019DC90E080E0DF91CF91FF90EF90DF906A
:10345000CF9008958DEE93E00CDCF3CF0F931F9384
:10346000CF93DF938C01D0E0C0E0CE010E94D10168
:10347000882319F0BE01C801B7DF2196C13ED105EE
:10348000A1F7DF91CF911F910F9108958FE094E004
:10349000F0DB88E092E0EDDB10DAECDB90E080E03E
:1034A00008954F925F926F927F928F929F92AF9208
:1034B000BF92CF92DF92EF92FF920F931F93CF9321
:1034C0006B017C01742EAC019B010E944457882340
:1034D00091F084E194E0CF911F910F91FF90EF90D4
:1034E000DF90CF90BF90AF909F908F907F906F9024
:1034F0005F904F9041CB46015701E894B7F82FEF0A
:103500003FEF4FE75FE7C501B4010E9444578111C7
:103510000DC02FEF3FEF4FE75FE7C501B4010E94F9
:10352000B35418161CF488E194E0D5CF2FEF3FEF89
:103530004FE75FE4C701B6010E94405718161CF41C
:103540008CE194E0C8CF2FEF3FEF4FE75FECC7016E
:10355000B6010E94B35487FDF3CF20E030E0A9010B
:10356000C701B6010E94B35410E000E087FF08C015
:103570008DE20E947A088C01F7FAF094F7F8F09443
:10358000C0E060E070E080E09FE37C1641F020E066
:1035900030E040E251E40E94A756CF5FF6CFA7018A
:1035A00096010E9443562B013C010E9414574B0187
:1035B0005C014AE0EEDA7C01E00EF11ECC23A9F1B9
:1035C000C501B4010E94B7549B01AC01C301B20113
:1035D0000E9442564B015C018EE20E947A08E80E7E
:1035E000F91EC15010F120E030E040E251E4C50185
:1035F000B4010E9418552B013C010E9414574B0145
:10360000B12CA12C4AE0C501B401C3DAE80EF91EC1
:10361000C501B4010E94B7549B01AC01C301B201C2
:103620000E9442564B015C01DCCFC701CF911F9134
:103630000F91FF90EF90DF90CF90BF90AF909F9051
:103640008F907F906F905F904F900895CF92DF9210
:10365000EF92FF92CF93DF93EC0188819981AA8149
:10366000BB81181619061A061B0644F081E090E08B
:10367000A0E0B0E088839983AA83BB838C819D817D
:10368000AE81BF81181619061A061B0644F081E0A8
:1036900090E0A0E0B0E08C839D83AE83BF838885FB
:1036A0009985AA85BB85181619061A061B0644F0CB
:1036B00081E090E0A0E0B0E088879987AA87BB8787
:1036C00080E294E0D6DA85E394E0D3DA60912E09C3
:1036D00070912F0980913009909131090E94B9545D
:1036E0006B017C01688179818A819B810E94B95438
:1036F0009B01AC01C701B6010E94A75642E0D1DE92
:1037000085E494E0B6DA60913209709133098091D2
:103710003409909135090E94B9546B017C016C8188
:103720007D818E819F810E94B9549B01AC01C701AC
:10373000B6010E94A75642E0B4DE85E594E099DA2E
:103740006091360970913709809138099091390953
:103750000E94B9546B017C01688579858A859B85B7
:103760000E94B9549B01AC01C701B6010E94A75643
:1037700042E097DEDF91CF91FF90EF90DF90CF9006
:1037800079CA9BD863DF90E080E008958F929F9282
:10379000AF92BF92CF92DF92EF92FF920F931F935F
:1037A000CF93DF93EC0186E292E063DA85E394E065
:1037B00060DA6E0184E6C81A8EEFD80AC6010E944C
:1037C000810F0E94B9544B015C01FE01EB54FD4F87
:1037D00060817181828193810E94B9549B01AC0107
:1037E000C501B4010E94A75642E05BDE85E494E087
:1037F00040DA7E01E4E3EE1AEEEFFE0AC7010E9412
:10380000810F0E94B9544B015C01FE01E754FD4F4A
:1038100060817181828193810E94B9549B01AC01C6
:10382000C501B4010E94A75642E03BDE85E594E065
:1038300020DA8E0104501E4FC8010E94810F0E94A1
:10384000B9544B015C01C354DD4F688179818A8191
:103850009B810E94B9549B01AC01C501B4010E9437
:10386000A75642E01EDE29D805DA82E292E001DAAC
:1038700085E394E0FED9F601A68DB78D20893189C4
:10388000428953890E940B56C7D985E494E0F1D947
:10389000F701A68DB78D20893189428953890E940D
:1038A0000B56BAD985E594E0E4D9F801A68DB78D19
:1038B00020893189428953890E940B56ADD90E94D3
:1038C0005D14DF91CF911F910F91FF90EF90DF90EA
:1038D000CF90BF90AF909F908F90CCC9CF92DF9246
:1038E000EF92FF920F931F93CF93DF938C016A01A6
:1038F0007B01EC01CC0FDD1F642FCE010E94D75558
:103900009927F7FC9A958F2D7E2D6D2DCE0101966E
:103910000E94D7550D5811090330110588F4B701DD
:10392000992777FD9095892FCE0144960E94D7550F
:103930006F2D772788279927CE0145960E94D75566
:1039400090E080E0DF91CF911F910F91FF90EF9079
:10395000DF90CF9008954F925F926F927F928F92F7
:103960009F92AF92BF92CF92DF92EF92FF920F930E
:103970001F93CF93DF938C01EC01CC0FDD1FCE01A1
:103980000E94CF55882E912CB12CA12CCE010196EE
:103990000E94CF55C82ED12CF12CE12C0D581109C5
:1039A0000330110508F05AC0CE0144960E94CF554D
:1039B000482E512C712C612CCE0145960E94CF557A
:1039C000082F10E030E020E08FEF4816510461042A
:1039D000710429F50F3F11052105310501F58FEF20
:1039E00088169104A104B104C9F58FEFC816D1045B
:1039F000E104F10499F56FEF7FEFCB01DF91CF91F7
:103A00001F910F91FF90EF90DF90CF90BF90AF90FC
:103A10009F908F907F906F905F904F9008950038A7
:103A20001105210531053CF7FE2CED2CDC2CCC24B6
:103A3000C701B601680D791D8A1D9B1D32015524F1
:103A40004424640D751D861D971D302F22271127D4
:103A50000027600F711F821F931FD0CF00E010E07E
:103A60009801412C512C320180E8C816D104E104A0
:103A7000F104D4F2C0CFEF92FF920F931F93CF9334
:103A8000DF938091140890911508892B51F584E0FB
:103A900090E00E943A4F7C0190E080E05CDF1616D7
:103AA000170654F1C7010E941914D0E0C0E0CE01FE
:103AB0000E94D101882369F0FE01EE0FFF1FEE0F77
:103AC000FF1FE75BF64F4081518162817381CE0118
:103AD00005DF2196C639D10551F7F0921508E0921D
:103AE00014088091140890911508DF91CF911F91CF
:103AF0000F91FF90EF90089583E090E02CDF61300C
:103B000071058105910531F509E419E0D0E0C0E0C7
:103B1000CE010E94D1018823B1F0CE011CDFF80153
:103B200060837183828393836F3F7F4F8F4F9F4F5B
:103B300051F4CE010E946702F801408151816281F7
:103B40007381CE01CBDE21960C5F1F4FC13ED105A4
:103B5000F9F6C3CFC7010E941914BFCF8CDF7EDCFA
:103B600084E294E086D80E945D1484D890E080E0DE
:103B70000895CF92DF92EF92FF920F931F93CF930E
:103B8000DF937C016B018A01E90175DFF601EE0F1D
:103B9000FF1FEE0FFF1FE75BF64F80819181F7015A
:103BA0009183808368DF000F111F000F111FF80140
:103BB000E75BF64F81E04081518162817381413042
:103BC00051056105710509F080E0F701828753DF37
:103BD000CC0FDD1FCC0FDD1FC75BD64F88819981CD
:103BE000AA81BB81F70182839383A483B583168264
:103BF000178210861186DF91CF911F910F91FF9050
:103C0000EF90DF90CF900895CF93DF93EC012AECF3
:103C100030E04BEC50E069EC70E0ABDF2EEC30E0D4
:103C20004FEC50E06DEC70E0CE010C96A2DF24ED7D
:103C300030E045ED50E063ED70E0CE01489699DF4D
:103C400028ED30E049ED50E067ED70E0CE0184965C
:103C500090DF2EED30E04FED50E06DED70E0CE01E5
:103C6000C096DF91CF9185CFCF93DF9380911B08D2
:103C700090911C08892BA1F48CE390E00E943A4FAC
:103C8000EC01198218821D861C86198E188E1DA2C1
:103C90001CA219AA18AAB8DFD0931C08C0931B084D
:103CA00080911B0890911C08DF91CF9108952F926D
:103CB0003F924F925F926F927F928F929F92AF92BC
:103CC000BF92CF92DF92EF92FF920F931F93CF9309
:103CD000DF93EC01D0DEFE01E551FD4F8091050B35
:103CE0009091060B91838083C6DEFE01E351FD4F68
:103CF0008091090B90910A0B91838083BCDEFE01B9
:103D0000E151FD4F80910D0B90910E0B91838083BB
:103D1000B2DE8E010F501D4F60912D0B70912E0B56
:103D200080912F0B9091300B0E94B954F801608361
:103D30007183828393839FDE1E01FBE02F1AFDEFC8
:103D40003F0A6091310B7091320B8091330B90914F
:103D5000340B0E94B954F101608371838283938391
:103D60008ADE20E030E048EC52E4F80160817181A5
:103D7000828193810E94A7562B013C0120E030E014
:103D800048EC52E4F10160817181828193810E944B
:103D9000A7564B015C016091350B7091360B8091F9
:103DA000370B9091380B0E94B95420E030E048EC7A
:103DB00052E40E94A7566B017C012AE037ED43E2F2
:103DC0005CE3C301B2010E94405718160CF02AC1EF
:103DD00020E030E046EC52E4C301B2010E94B3544B
:103DE00087FD06C0412C512C56EC652E52E4752EF1
:103DF000F80140825182628273822AE037ED43E209
:103E00005CE3C501B4010E94405718160CF013C1C1
:103E100020E030E046EC52E4C501B4010E94B35406
:103E200087FD06C0812C912C36ECA32E32E4B32EF4
:103E3000F10180829182A282B3822AE037ED43E2CF
:103E40005CE3C701B6010E94405718160CF0FCC095
:103E500020E030E046EC52E4C701B6010E94B354C2
:103E600087FD06C0C12CD12C96ECE92E92E4F92EE8
:103E7000FE01E750FD4FC082D182E282F382FBDD7A
:103E80008091ED0A9091EE0AFE01FD5F918380839F
:103E9000F2DD8091F10A9091F20AFE01EE5FFC4F93
:103EA00091838083E8DD8091F50A9091F60AFE0106
:103EB000EC5FFC4F91838083DEDD8091150B909148
:103EC000160BA091170BB091180BFE01EA5FFC4F87
:103ED00080839183A283B383CEDD8091190B90916F
:103EE0001A0BA0911B0BB0911C0BFE01E65FFC4F5F
:103EF00080839183A283B383BEDD80911D0B90915B
:103F00001E0BA0911F0BB091200BFE01E25FFC4F36
:103F100080839183A283B383AEDD80913D0B90912A
:103F20003E0BFE01EE5EFC4F91838083A4DD809109
:103F3000410B9091420BFE01EC5EFC4F918380831C
:103F40009ADD8091450B9091460BFE01EA5EFC4F95
:103F50009183808390DD8091550B9091560BFE01EB
:103F6000E85EFC4F9183808386DD8091590B9091B0
:103F70005A0BFE01E65EFC4F918380837CDD8091CD
:103F80005D0B90915E0BFE01E45EFC4F918380839C
:103F900072DD8091DD0A9091DE0AA091DF0AB09176
:103FA000E00AFE01E350FD4F0197A105B10509F0BC
:103FB00054C081E080835FDD8091E10A9091E20A44
:103FC000A091E30AB091E40AFE01E250FD4F01978F
:103FD000A105B10509F043C081E080834CDD8091EB
:103FE000E50A9091E60AA091E70AB091E80AC1506B
:103FF000DD4F0197A105B105A1F581E08883DF912F
:10400000CF911F910F91FF90EF90DF90CF90BF90D5
:10401000AF909F908F907F906F905F904F903F9068
:104020002F9008954AE0442E47ED542E43E2642E2B
:104030004CE3742EDDCE2AE0822E27ED922E23E271
:10404000A22E2CE3B22EF4CE8AE0C82E87EDD82E15
:1040500083E2E82E8CE3F82E0BCF1082ACCF1082D7
:10406000BDCF1882CCCF2F923F924F925F926F922A
:104070007F928F929F92AF92BF92CF92DF92EF92F8
:10408000FF920F931F93CF93DF93CDB7DEB7659762
:104090000FB6F894DEBF0FBECDBF998B888BEBDCDB
:1040A000E889F989ED5BFD4F81E04091150A509157
:1040B000160A6091170A7091180A452B462B472B58
:1040C00009F480E08083D7DCE889F989EC5BFD4F57
:1040D00081E04091190A50911A0A60911B0A70916F
:1040E0001C0A452B462B472B09F480E08083C3DC58
:1040F000E889F989EB5BFD4F81E040911D0A509101
:104100001E0A60911F0A7091200A452B462B472BEF
:1041100009F480E08083AFDC8091650A9091660AA3
:10412000A091670AB091680AE889F989EA5BFD4FB6
:1041300080839183A283B3839EDC8091690A9091EE
:104140006A0AA0916B0AB0916C0AE889F989E65B6A
:10415000FD4F80839183A283B3838DDC80916D0AB0
:1041600090916E0AA0916F0AB091700AE889F9895E
:10417000E25BFD4F80839183A283B3837CDC8091DB
:104180003D0A90913E0AA0913F0AB091400AE88909
:10419000F989E25AFD4F80839183A283B3836BDC5C
:1041A0008091410A9091420AA091430AB091440A39
:1041B000E889F989EE59FD4F80839183A283B38307
:1041C0005ADC8091450A9091460AA091470AB09125
:1041D000480AE889F989EA59FD4F80839183A283CF
:1041E000B38349DC80914D0A90914E0AA0914F0A09
:1041F000B091500AE889F989E659FD4F808391838F
:10420000A283B38338DC8091510A9091520AA09125
:10421000530AB091540AE889F989E259FD4F808325
:104220009183A283B38327DC8091550A9091560A2B
:10423000A091570AB091580AE889F989EE58FD4FC4
:1042400080839183A283B38316DC8091ED099091E2
:10425000EE09A091EF09B091F009E889F989EA58CF
:10426000FD4F80839183A283B38305DC8091F109A4
:104270009091F209A091F309B091F409E889F989C4
:10428000E658FD4F80839183A283B383F4DB809152
:10429000F5099091F609A091F709B091F809E8891C
:1042A000F989E258FD4F80839183A283B383E3DBD6
:1042B000E889F989EE57FD4F81E02091C5093091D9
:1042C000C6092130310509F080E08083D4DBE8891C
:1042D000F989ED57FD4F81E02091C9093091CA0954
:1042E0002130310509F080E08083C5DBE889F98958
:1042F000EC57FD4F81E02091CD093091CE0921305E
:10430000310509F080E08083B6DBE889F989E05661
:10431000FD4F81E040919D0950919E0960919F0958
:104320007091A009452B462B472B09F480E0808330
:10433000A2DBE889F989EF55FD4F81E04091A109A1
:104340005091A2096091A3097091A409452B462BB5
:10435000472B09F480E080838EDBE889F989EE55EC
:10436000FD4F81E04091A5095091A6096091A709F0
:104370007091A809452B462B472B09F480E08083D8
:104380007ADBE889F989ED55FD4F81E04091750AA6
:104390005091760A6091770A7091780A452B462BE6
:1043A000472B09F480E0808366DBE889F989EC55C6
:1043B000FD4F81E04091790A50917A0A60917B0A21
:1043C00070917C0A452B462B472B09F480E08083B3
:1043D00052DBE889F989EB55FD4F81E040917D0A78
:1043E00050917E0A60917F0A7091800A452B462B7E
:1043F000472B09F480E080833EDBE889F989EA55A0
:10440000FD4F81E02091AD093091AE092130310599
:1044100009F080E080832FDBE889F989E955FD4FB9
:1044200081E02091B1093091B2092130310509F0C4
:1044300080E0808320DBE889F989E855FD4F81E041
:104440002091B5093091B6092130310509F080E09D
:10445000808311DB8091750990917609A09177098D
:10446000B0917809E889F989E755FD4F80839183F8
:10447000A283B38300DB8091790990917A09A0919E
:104480007B09B0917C09E889F989E355FD4F808368
:104490009183A283B383EFDA80917D0990917E09A5
:1044A000A0917F09B0918009E889F989EF54FD4F07
:1044B00080839183A283B383DEDAE889F989EC569D
:1044C000FD4F81E0409185095091860960918709EF
:1044D00070918809452B462B472B09F480E0808397
:1044E000CADAE889F989EB56FD4F81E040918909E4
:1044F00050918A0960918B0970918C09452B462B4C
:10450000472B09F480E08083B6DAE889F989EA5616
:10451000FD4F81E040918D0950918E0960918F0986
:1045200070919009452B462B472B09F480E080833E
:10453000A2DA80917D0B90917E0BA0917F0BB091C0
:10454000800BE889F989EB57FD4F80839183A28323
:10455000B38391DA8091810B9091820BA091830BB0
:10456000B091840BE889F989E757FD4F80839183E7
:10457000A283B38380DA8091850B9091860BA09102
:10458000870BB091880BE889F989E357FD4F808349
:104590009183A283B3836FDAE889F989E956FD4FE5
:1045A00081E02091DD093091DE092130310509F0EB
:1045B00080E08083E889F989E856FD4F1082E88918
:1045C000F989E756FD4F108256DAE889F989E656EF
:1045D000FD4F81E02091D9093091DA092130310570
:1045E00009F080E08083E889F989E556FD4F108263
:1045F000E889F989E456FD4F10823DDAE889F989A6
:10460000E356FD4F81E02091FD093091FE092130F4
:10461000310509F080E080832EDAE889F989E256D5
:10462000FD4F81E02091010A3091020A21303105CD
:1046300009F080E080831FDAE889F989E156FD4FAF
:1046400081E02091050A3091060A2130310509F0F8
:1046500080E0808310DAE889F989EF56FD4F81E028
:1046600020918D0B30918E0B2130310509F080E0C7
:10467000808301DAE889F989EE56FD4F81E02091C7
:10468000910B3091920B2130310509F080E080834D
:10469000F2D9E889F989ED56FD4F81E02091950B1B
:1046A0003091960B2130310509F080E08083E3D909
:1046B000088919890B541D4F8091250A9091260A6B
:1046C000A091270AB091280AF80180839183A283E0
:1046D000B383D1D9E888F988F7E4EF1AFDEFFF0A30
:1046E0008091290A90912A0AA0912B0AB0912C0A54
:1046F000F70180839183A283B383BDD980912D0A72
:1047000090912E0AA0912F0AB091300AC888D988BA
:10471000F3E4CF1AFDEFDF0AF60180839183A283D1
:10472000B383F801408151816281738114161506AB
:104730001606170644F041E050E060E070E0408368
:10474000518362837383F701408151816281738158
:10475000141615061606170644F041E050E060E016
:1047600070E04083518362837383181619061A061A
:104770001B064CF081E090E0A0E0B0E0F601808301
:104780009183A283B3830E945D14FC01D6018D90B6
:104790009D90AD90BC90D7014D915D916D917C91B4
:1047A000D8010D911D912D913C910083118322839D
:1047B0003383448355836683778380869186A2867C
:1047C000B386E889F9897096FB83EA83E889F989D9
:1047D000EF56FD4F20812983E889F989EB57FD4F7A
:1047E00080819181A281B381E889F989E356FD4FE7
:1047F00020812D83E889F989EA55FD4F20812C839A
:10480000E889F989E956FD4F20812987E889F989E6
:10481000E656FD4F20812A87E889F989ED55FD4F3D
:1048200020812E87E889F989E056FD4F20812F8766
:10483000E889F989EE57FD4F2080E889F989ED5B19
:10484000FD4F3080E889F989E755FD4F408151815E
:1048500062817381E889F989EA58FD4F00811181ED
:1048600022813381E889F989E659FD4FC080D180E2
:10487000E280F380E889F989E25AFD4F80809180D7
:10488000A280B380E889F989EA5BFD4F40805180BE
:1048900062807380E889F98946A657A660AA71AA42
:1048A00082AA93AAA4AAB5AAC6AAD7AAE0AEF1AED4
:1048B00002AF13AF24AF35AFFE96408351836283BE
:1048C0007383E889F989EE5BFF4F3082E889F989C3
:1048D000ED5BFF4F20822F85E889F98923A72E857C
:1048E00024A72C8125A740E450E060E070E0EA5B5B
:1048F000FF4F4083518362837383E889F989EC5BBE
:10490000FF4F2A852083E889F989EB5BFF4F2985D2
:104910002083E889F989E65BFF4F2D812083E889B0
:10492000F989E55BFF4F80839183A283B383E88994
:10493000F989E15BFF4F89818083A889B9895B96FA
:104940008D919C915C978633910509F034C286E481
:104950009CE0FD01EC57FF4F9183808332961182DA
:10496000108284E49CE03696918380833296118293
:104970001082E889F98981A192A14A97D1F482E451
:104980009CE0E857FF4F91838083E889F989E657D7
:10499000FF4F1182108280E49CE0E889F989E0579A
:1049A000FF4F91838083E889F989EE56FF4F11828A
:1049B0001082088919890C561F4FE889F989EE562B
:1049C000FD4F20812983E889F989E757FD4F8081D0
:1049D0009181A281B3818D839E83AF83B887E8895B
:1049E000F989E256FD4F90819C83E889F989E95560
:1049F000FD4FA081A987E889F989E856FD4FB0816C
:104A0000BA87E889F989E556FD4F20812E87E88924
:104A1000F989EC55FD4F2080E889F989EF55FD4F64
:104A20003080E889F989ED57FD4F3081E889F989AF
:104A3000EC5BFD4F2081E889F989E355FD4F8081CA
:104A40009181A281B381E889F989E658FD4F4081BF
:104A5000518162817381E889F989E259FD4FC080F3
:104A6000D180E280F380E889F989EE59FD4F80809A
:104A70009180A280B380E889F989E65BFD4F408090
:104A8000518062807380F801468E578E60A271A2B9
:104A900082A293A2A4A2B5A2C6A2D7A2E0A6F1A622
:104AA00042A753A764A775A786A797A7A0ABB1ABEA
:104AB00022AB33AB338E248E2985258F80E490E0A2
:104AC000A0E0B0E086AB97ABA0AFB1AF2E8524AB32
:104AD0008A8585AB9C8192AF8D819E81AF81B8859F
:104AE00083AF94AFA5AFB6AF298127AF83859485F7
:104AF0008633910509F091C186E49CE0E889F98943
:104B0000E85FFE4F91838083E889F989E65FFE4F75
:104B10001182108284E49CE0E889F989E05FFE4F0D
:104B200091838083E889F989EE5EFE4F11821082BD
:104B3000D80151968D919C914A97E1F482E49CE0D2
:104B4000E889F989E45FFE4F91838083E889F989D8
:104B5000E25FFE4F1182108280E49CE0E889F989CF
:104B6000EC5EFE4F91838083E889F989EA5EFE4F0F
:104B700011821082E888F988B8EEEB1ABEEFFB0AC2
:104B8000E889F989ED56FD4F20812983E889F98963
:104B9000E357FD4F80819181A281B3818D839E83F4
:104BA000AF83B887E889F989E156FD4F90819C83EE
:104BB000E889F989E855FD4F3080E889F989E75699
:104BC000FD4FA081A987E889F989E456FD4F20802F
:104BD000E889F989EB55FD4FC080E889F989EE55E0
:104BE000FD4FD080E889F989EC57FD4F3081E88985
:104BF000F989EB5BFD4F2081E889F989EF54FD4F7E
:104C000080819181A281B3818A8B9B8BAC8BBD8B80
:104C1000E889F989E258FD4F4081518162817381B1
:104C2000E889F989EE58FD4F80809180A280B38099
:104C3000E889F989EA59FD4F40805180628073808C
:104C4000E889F989E25BFD4F80819181A281B3817E
:104C5000F701868F978FA0A3B1A342A253A264A2AB
:104C600075A286A297A2A0A6B1A642A753A764A741
:104C700075A78A899B89AC89BD8986A797A7A0ABB0
:104C8000B1AB22AB33ABD38EC48E358E80E490E0D3
:104C9000A0E0B0E086AB97ABA0AFB1AF24AA298566
:104CA00025AB8C8182AF8D819E81AF81B88583AF2A
:104CB00094AFA5AFB6AF298127AF8385948586339E
:104CC000910509F0D2C086E49CE0E889F989E457AF
:104CD000FE4F91838083E889F989E257FE4F118264
:104CE000108284E49CE0E889F989EC56FE4F9183B8
:104CF0008083E889F989EA56FE4F11821082D70134
:104D000051968D919C914A97E1F482E49CE0E88968
:104D1000F989E057FE4F91838083E889F989EE563F
:104D2000FE4F1182108280E49CE0E889F989E85600
:104D3000FE4F91838083E889F989E656FE4F118200
:104D40001082E889F989EC56FD4F8081882309F4A7
:104D5000B4C08A819B810E94CD0CE889F989EB5609
:104D6000FD4F8081882309F4ADC0C8010E94CD0C9D
:104D7000E889F989EA56FD4F8081882309F4A6C0A5
:104D8000C70165960FB6F894DEBF0FBECDBFDF91A9
:104D9000CF911F910F91FF90EF90DF90CF90BF9038
:104DA000AF909F908F907F906F905F904F903F90CB
:104DB0002F900C94CD0C8C339105D9F48EE39CE0AC
:104DC000E889F989EC57FF4F91838083E889F98955
:104DD000EA57FF4F118210828CE39CE0E889F98941
:104DE000E457FF4F91838083E889F989E257FF4FA9
:104DF000BECD8E9709F0BDCD86E39CE0E889F989A8
:104E0000EC57FF4F91838083E889F989EA57FF4F78
:104E10001182108280E39CE0E1CF8C33910589F40C
:104E20008EE39CE0E889F989E85FFE4F91838083F7
:104E3000E889F989E65FFE4F118210828CE39CE0DD
:104E40006BCE8E9709F074CE86E39CE0E889F989F1
:104E5000E85FFE4F91838083E889F989E65FFE4F22
:104E60001182108280E39CE057CE8C33910589F447
:104E70008EE39CE0E889F989E457FE4F91838083B3
:104E8000E889F989E257FE4F118210828CE39CE099
:104E90002ACF8E9709F033CF86E39CE0E889F98921
:104EA000E457FE4F91838083E889F989E257FE4FEA
:104EB0001182108280E39CE016CF8A819B810E9440
:104EC000BB0C4BCFC8010E94BB0C52CFC7016596EB
:104ED0000FB6F894DEBF0FBECDBFDF91CF911F910B
:104EE0000F91FF90EF90DF90CF90BF90AF909F9089
:104EF0008F907F906F905F904F903F902F900C9489
:104F0000BB0CAF92BF92CF92DF92EF92FF920F93C2
:104F10001F93CF93DF93EC018AE190E09C8F8B8FFE
:104F20008BE190E09E8F8D8F89E190E098A38F8F29
:104F30008FE090E09AA389A38EE190E09CA38BA3DD
:104F40008EE090E09EA38DA385E490E098A78FA3C8
:104F500084E490E09AA789A7FE01EC56FF4F80E217
:104F600090E09487838781E290E0968785878FE140
:104F700090E0908B8787128A118A148A138A168A86
:104F8000158A83E490E0908F878B82E490E0928F83
:104F9000818FEC57FF4F83E290E09487838784E210
:104FA00090E09687858782E290E0908B8787128ACF
:104FB000118A148A138A168A158A81E490E0908FE8
:104FC000878B80E490E0928F818FEB5DFE4F1182A2
:104FD0001082329611821082329611821082CE0196
:104FE00042D8CE010E94571ECE0184569E4F41E00A
:104FF00050E0FC0157A746A7DE01A453BE4F24E0B2
:1050000030E09F963C932E939E975E01F4E0AF1A9A
:10501000FEEFBF0A28E030E0F50137A726A720E120
:1050200030E0FC013183208321E130E035832483AB
:105030002FEF3FEF33832283378326836285608798
:105040006385618767E170E011967C936E9368E1F8
:1050500070E015967C936E93149713963C932E9361
:10506000129717963C932E9316971A966C911A974F
:1050700018966C9318971B966C911B9719966C93C6
:1050800019976DE170E0F501718360836CE170E068
:1050900075836483338322833783268362856087A5
:1050A00063856187BE01685E7C4FFB016081718111
:1050B0008E010A5F1C4FF801C080D180E280F3802E
:1050C00006501109F80100811181FC01158F048F30
:1050D000C48AD58AE68AF78A6130710509F04EC024
:1050E000378F268FCE01865E9C4FFC018081918197
:1050F0009E01265F3C4FF90140815181628173819D
:1051000028503109F901208131815D963C932E931D
:105110005C9754964D935D936D937C93579701974D
:1051200081F58FEF9FEF5F969C938E935E97DE01E4
:10513000A45EBC4F8D919C9111971E974D915D91EE
:105140006D917C91CC5FDC4F28813981F501358FE1
:10515000248F448B558B668B778B0197A9F48FEF47
:105160009FEF978F868FDF91CF911F910F91FF90C7
:10517000EF90DF90CF90BF90AF900895578F468FFC
:10518000B1CF81E090E0CFCF81E090E0EACF2F92E5
:105190003F924F925F926F927F928F929F92AF92C7
:1051A000BF92CF92DF92EF92FF920F931F93CF9314
:1051B000DF9300D01F92CDB7DEB79C838B830E9414
:1051C0003B1D60908D0A70908E0A0E943B1D80905E
:1051D0009D0A90909E0A0E943B1D2090B50A309037
:1051E000B60A0E943B1DC090910AD090920A0E947C
:1051F0003B1DA090A10AB090A20A0E943B1D4090C6
:10520000B90A5090BA0A0E943B1D0091950A10916C
:10521000960A0E943B1DE090A50AF090A60A0E9403
:105220003B1D8091BD0A89838091BE0A8A839101CA
:105230001216130614F021E030E0A401B3018B81B3
:105240009C8140960E94EB1292011414150414F0F4
:1052500021E030E0A501B6018B819C818C569F4FE7
:105260000E94EB1229813A811216130614F021E0F4
:1052700030E0A701B8018B819C81885E9E4F0F9022
:105280000F900F900F90DF91CF911F910F91FF9092
:10529000EF90DF90CF90BF90AF909F908F907F90D6
:1052A0006F905F904F903F902F900C94EB12CF92A5
:1052B000DF92EF92FF920F931F93CF93DF938B01B7
:1052C0000E943B1DEC01F801C2A0D3A0E4A0F5A010
:1052D000068D178D8A819B818F30F7E29F075CF5E1
:1052E00001969B838A83C8010E94D101882331F1F2
:1052F000F801EE0FFF1FEE0FFF1FE75BF64FC082B6
:10530000D182E282F382B701A601C8010E946E1C1D
:10531000B801CE010E94F4190E94341E0E94041E9E
:1053200090E080E0DF91CF911F910F91FF90EF907F
:10533000DF90CF9008951B821A82D5CF8DEE93E037
:105340000E943916E9CFCF93DF93EB010E943B1DFA
:105350006E8D7F8D0E94F41990E080E0DF91CF91F7
:105360000895FC0180819181009711F00C94D64F33
:1053700008950C94D64F0C94D64F0C94D64F0C94A1
:10538000D64F0C94D64F0C94D64F0C94D64F0C9409
:10539000D64F0C94D64F0C94D64F0C94D64F0C94F9
:1053A000D64F0C94D64F0C94D64F0C94D64F0C94E9
:1053B000D64F0C94D64F0C94D64F0C94D64F0C94D9
:1053C000D64F0C94D64F0C94D64F0C94D64F0F93C7
:1053D0001F93CF93DF93EC0188819981009759F057
:1053E0002A813B812617370730F081E0DF91CF918A
:1053F0001F910F9108958B016F5F7F4F0E946B5734
:10540000009759F0998388831B830A832C813D81FF
:10541000232B59F7FC011082E8CF80E0E7CF0F93F0
:105420001F93CF93DF93EC018B01D1DF288139816A
:10543000811112C02115310519F0C9010E94D64F02
:10544000198218821D821C821B821A82CE01DF9172
:10545000CF911F910F9108951D830C8360EE77E02B
:10546000C9010E945C58F2CF70E060E0D8CF2F9263
:105470003F924F925F926F927F928F929F92AF92E4
:10548000BF92CF92DF92EF92FF920F931F93CF9331
:10549000DF93CDB7DEB7C458D1090FB6F894DEBF9D
:1054A0000FBECDBF8C01FC011082118212821382CB
:1054B0001482158216821782108611861286138630
:1054C00014861586168617864C01F0E18F0E911C06
:1054D000C4010E94B20E580184E9A80EB11CC50196
:1054E0000E94B20E6801E8EECE1AEEEFDE0AC601A7
:1054F0000E94B20E7801F4E6EF1AFEEFFF0AC70130
:105500000E94E30F380184E3681A8EEF780AC30122
:105510000E94E30F2801E4E04E1AEEEF5E0AC2019A
:105520000E94E30FF801E45DFD4F118210821382A7
:10553000128215821482CF0197DFF801EE5CFD4FD5
:10554000118210823296118210823296118210825C
:1055500032961182108232961082319610823196E4
:105560001082319611821082329611821082329608
:1055700011821082329610823196108231961082FA
:105580003196108211821282138234961082118217
:105590001282138234961082118212821382349600
:1055A000108211821282138234961082118212822A
:1055B00013823496108211821282138234961082E2
:1055C0001182128213823496108211821282138207
:1055D00034961082118212821382349610821182C4
:1055E00012821382349610821182128213823496B0
:1055F00010821182128213823496108211821282DA
:105600001382349610821182128213823496108291
:105610001182128213823496108231961082319652
:105620001082319610821182128213823496108277
:105630001182128213823496108211821282138296
:1056400034961082319610823196108231961082F3
:1056500031961082319610823196108231961082E6
:1056600031961082319610823196108231961082D6
:1056700031961082319610823196108231961082C6
:1056800031961082319610823196108231961082B6
:1056900031961082319610823196108231961082A6
:1056A00031961082118212821382349610821182F6
:1056B0001282138234961082118212821382D801D0
:1056C000AB54BD4F8CE0E1E1F2E001900D928A9580
:1056D000E1F7F801EF53FD4F10821182128213821D
:1056E00034961082118212821382349610821182B3
:1056F00012821382349611821082329611821082A5
:105700003296118210823296108211821282138296
:105710003496108211821282138234961082118282
:10572000128213823496108211821282138234966E
:105730001082118212821382349610821182128298
:105740001382349611821082329611821082329620
:105750001182108232961082118212821382349644
:105760001082118212821382349610821182128268
:1057700013823496108231961082319610823196BF
:10578000118210823296118210823296118210821A
:105790003296108211821282138234961082118204
:1057A00012821382349610821182128213823496EE
:1057B00011821082329611821082329611821082EA
:1057C00032961182108232961182108232961182A4
:1057D0001082329611821082329611821082180144
:1057E000FEED2F1AFCEF3F0AF10110823196118273
:1057F0001082329611821082CE0101960E94B20E62
:1058000084E8FE013196D40101900D928A95E1F76A
:10581000CE0101960E94B20E84E8FE013196D501B8
:1058200001900D928A95E1F7CE0101960E94B20E89
:1058300084E8FE013196D60101900D928A95E1F738
:1058400088E5F801848BE856FF4F89E58083EC57A3
:10585000FF4F8AE58083CE0101960E94E30F80E32B
:10586000FE013196D70101900D928A95E1F7CE01A4
:1058700001960E94E30F80E3FE013196D30101906F
:105880000D928A95E1F7CE0101960E94E30F80E325
:10589000FE013196D20101900D928A95E1F7C8017F
:1058A00030DBF1011082CC57DF4F0FB6F894DEBF2A
:1058B0000FBECDBFDF91CF911F910F91FF90EF9061
:1058C000DF90CF90BF90AF909F908F907F906F9020
:1058D0005F904F903F902F900895CF93DF938091EA
:1058E000120890911308892B51F487E293E00E94EB
:1058F0003A4FEC01BCDDD0931308C093120880919D
:10590000120890911308DF91CF910895CF93DF9300
:1059100080911808811114C081E080931808DDDFA0
:10592000EC0140960E947E0ECE018C569F4F0E9445
:105930007E0ECE01885E9E4F0E947E0E1092180849
:10594000DF91CF910895CF93DF93EB0120E030E01A
:1059500040E85FE36A817B818C819D810E94B35422
:1059600081110CC088E294E00E943916B6DF8C5A8F
:105970009F4FFC01108211821282138220E030E0DE
:1059800040E85FE36E817F81888599850E94B354EA
:1059900081110CC088E394E00E9439169EDF885282
:1059A0009F4FFC01108211821282138220E030E0AE
:1059B00040E85FE36A857B858C859D850E94B354B2
:1059C00081110CC088E494E00E94391686DF845A65
:1059D0009E4FFC0110821182128213820E945D147C
:1059E0000E943A1690E080E0DF91CF910895CF9326
:1059F000DF93FC01E05DFD4F408151814115510570
:105A000001F1EC01CC5CDD4F28813981845D9D4F33
:105A100024173507E8F4FC01808191810097A1F0FB
:105A2000820F931FFC0180818A3031F08D3069F440
:105A30008EED97E00E9439168881998101969983AD
:105A40008883DF91CF91089580E00E947A08F4CF97
:105A500070E060E0E4DC19821882F3CFEF92FF92ED
:105A60000F931F93CF93DF936115710541F480E08D
:105A7000DF91CF911F910F91FF90EF900895411505
:105A80005105A9F07B01EC010C811D81040F151F4C
:105A9000B8019DDC882359F3288139818C819D814F
:105AA000B701820F931F0E945C581D830C8381E015
:105AB000DFCFEF92FF920F931F93CF93DF93CDB77A
:105AC000DEB764970FB6F894DEBF0FBECDBF7C0182
:105AD000CB01BA018E010F5F1F4F22E044E00E940C
:105AE0001D4FFC0101900020E9F73197AF01481BE1
:105AF000590BBC01C701B2DF64960FB6F894DEBF44
:105B00000FBECDBFDF91CF911F910F91FF90EF900E
:105B10000895EF92FF920F931F93CF93DF9300D0DE
:105B200000D01F92CDB7DEB77C01CB014AE08E01D9
:105B30000F5F1F4FB8010E94C550F801019000206F
:105B4000E9F73197AF01401B510BB801C70186DF60
:105B500027960FB6F894DEBF0FBECDBFDF91CF9171
:105B60001F910F91FF90EF900895FB01019000208D
:105B7000E9F73197AF01461B570B70CFEF92FF92B9
:105B80000F931F93CF93DF93CDB7DEB72E970FB64A
:105B9000F894DEBF0FBECDBF8C01FC0111821082D4
:105BA00013821282158214825FDC68E873E0C801F8
:105BB000DCDF6091CD0C7091CE0C8091CF0C909178
:105BC000D00C2AE0AE014F5F5F4F7A010E949650E1
:105BD000F70101900020E9F73197AF014E195F09F5
:105BE000B701C8013BDF6EED77E0C801BEDFC80139
:105BF0002E960FB6F894DEBF0FBECDBFDF91CF91CA
:105C00001F910F91FF90EF900895FB014481558102
:105C10006081718123CFCF92DF92EF92FF920F9339
:105C20001F93CF93DF9300D000D01F921F92CDB768
:105C3000DEB78B016A01845D9D4F7C016AE272E0F0
:105C400094DF62E174E0C70190DFF8018481898309
:105C50001A8241E050E08E010F5F1F4FB801C7016B
:105C6000FDDE4AE0B801C6010E948C50F8010190A7
:105C70000020E9F73197AF01401B510BB801C70174
:105C8000EDDE0E945D14C80179DFB801C701BDDFF8
:105C9000C80167DB28960FB6F894DEBF0FBECDBFF4
:105CA000DF91CF911F910F91FF90EF90DF90CF90F8
:105CB00008952F923F924F925F926F927F928F92B0
:105CC0009F92AF92BF92CF92DF92EF92FF920F938B
:105CD0001F93CF93DF93CDB7DEB7A1970FB6F8949C
:105CE000DEBF0FBECDBF99A388A3798768870E94C6
:105CF000332088A199A10E94571E0E94E6140E9499
:105D0000D01928853985C8A0D9A02130310509F4DA
:105D100062C02230310509F48EC030E1C30ED11CBF
:105D200048A159A144565E4F5A834983E8A1F9A17D
:105D3000E056FD4F50815D8388A199A18F539D4FFF
:105D40009C838B83E8A1F9A1E551FD4FF98BE88B8A
:105D500028A139A123503D4F3D8B2C8B48A159A13F
:105D6000435C5D4F5F834E838DE890E09B8B8A8B15
:105D7000E5E1F0E0FD87EC87C6010E94800C8823F6
:105D800009F488C088E594E00E9439160E945D14E9
:105D900081E090E090935E0880935D082224239434
:105DA000312CC101A1960FB6F894DEBF0FBECDBF56
:105DB000DF91CF911F910F91FF90EF90DF90CF90E7
:105DC000BF90AF909F908F907F906F905F904F901B
:105DD0003F902F900895F4E9CF0ED11C28A139A14E
:105DE00024533E4F3A832983E8A1F9A1EF55FD4F93
:105DF00030813D8348A159A14B535D4F5C834B8358
:105E000088A199A183519D4F998B888BE8A1F9A115
:105E1000E250FD4FFD8BEC8B28A139A1215C3D4F59
:105E20003F832E834EE850E05B8B4A8B86E190E007
:105E30009D878C87A1CF98EEC91A9EEFD90AE8A159
:105E4000F9A1E450FE4FFA83E983E8A1F9A1EE55E8
:105E5000FD4F20812D8348A159A147535D4F5C839D
:105E60004B8388A199A181519D4F998B888BE8A183
:105E7000F9A1E150FD4FFD8BEC8B28A139A12F5BDF
:105E80003D4F3F832E834FE850E05B8B4A8B87E189
:105E900090E0CECFC6010E94710C811173CF81E9D1
:105EA00093E00E9439168EE894E00E943916F601BC
:105EB00084810E947A0885E994E00E9439168EED6B
:105EC00097E00E94391681E090E0EE81FF81918396
:105ED000808341E050E0B60188A199A19CDEC60113
:105EE0000E94CD0CF60182A9860106591F4F882316
:105EF00009F4A5C0C6010E948F0CF80110828981A7
:105F00009A810E94810FF601EC5BFF4F60837183E1
:105F100082839383EB81FC8110821182128213822F
:105F2000E8A1F9A1EF53FD4F108211821282138272
:105F3000E8A1F9A1EB53FD4F108211821282138266
:105F4000E8A1F9A1E753FD4F10821182128213825A
:105F500086E090E0EE81FF819183808346E050E00F
:105F6000B60188A199A157DE61E070E0C6010E94E8
:105F7000511628853985220F331F220F331F3B8787
:105F80002A87C9018F509D4F48A159A1480F591F19
:105F90005B8F4A8F4E97E8A1F9A1E80FF91FFD8F9B
:105FA000EC8F429728A139A1280F391F3F8F2E8FE0
:105FB000812C912C540183948885998583509D4F21
:105FC00048A159A1480F591F598F488F2A843B84F3
:105FD00088A199A1280E391EF101E659FD4FFF8BCA
:105FE000EE8B60E5462E63EC562E612C712CE88C0E
:105FF000F98C0A8D1B8D2C8D3D8D4E8D5F8D6981A9
:106000007A81C6010E94EE1081ED9CE00E94F707A4
:1060100018161906DCF010E0312C212CC6010E9464
:10602000800C882389F189EC94E00E943916C6011E
:106030000E94800C811101C08D818D8387C0C601B3
:106040000E94A50C81E0F801808359CF81ED9CE08E
:106050000E94D5078F7D85349105E9F684EB94E0A5
:106060000E9439160E945D1421E0FC01268786E516
:1060700092E00E9439160E945D140E943A16222472
:106080002394312C11E0CACFC6010E94710C8111FA
:10609000CACF1111C8CFE889F98960817181072EB3
:1060A000000C880B990B0E94B9549B01AC01EB8149
:1060B000FC8160817181828193810E94B35487FF4A
:1060C000B2CFC6010E94770DEE89FF892081318110
:1060D00042815381C301B2010E94E555C9010E946A
:1060E000030AEE89FF892081318142815381A3E037
:1060F000B0E00E9401569B01AC01C501B4010E94B1
:10610000E555672B682B692B41F482E592E00E94EC
:1061100039160E945D140E943A16C6010E94580C5E
:10612000EE89FF892081318142815381C301B2010F
:106130000E94E555C9010E94030AFFEF8F1A9F0ACA
:10614000AF0ABF0A2114310409F451CF62E070E0B4
:10615000C6010E94511681E993E00E9439168EE82B
:1061600094E00E943916F60184810E947A088DED30
:1061700094E00E9439168EED97E00E9439162114A2
:10618000310409F580EF94E00E94391682E194E031
:106190000E9439168FE893E00E9439168C859D8500
:1061A0000E94341682E194E00E9439168FE098E054
:1061B0000E943916FD818F2F90E00E9434160E94B4
:1061C0005D140E943A160E94E6140E94D01981E9DB
:1061D00093E00E9439168EE894E00E943916F60189
:1061E00084810E947A0884EF94E00E9439168EED33
:1061F00097E00E943916EB81FC8110821182128295
:106200001382F60182A9860106591F4F882309F4DB
:106210000EC1C6010E94A50C81E0F801808389812E
:106220009A810E94810FF601EC5BFF4F60837183BE
:1062300082839383E8A1F9A1EF53FD4F108211826D
:1062400012821382E8A1F9A1EB53FD4F1082118253
:1062500012821382E8A1F9A1E753FD4F1082118247
:106260001282138289819A810E94810F6C877D87B7
:106270008E879F8789819A810E94810F412C512CA2
:106280003201AA84BB8428A139A1A20EB31E36E92B
:10629000A31A3DEFB30A42012114310469F5E88CD9
:1062A000F98C0A8D1B8D2C8D3D8D4E8D5F8D6981F6
:1062B0007A81C6010E94EE1081ED9CE00E94F707F2
:1062C000181619060CF4B9C010E03AE083169104D0
:1062D00034F4EB81FC811082118212821382FD81E1
:1062E000C601F1114CC10E94800C882309F4C4C07E
:1062F00089EC94E00E94391681E993E00E943916F6
:106300008EE894E00E943916F60184810E947A0892
:1063100086E195E00E9439168EED97E00E943916CD
:1063200089819A810E94810F2C893D89232BA1F0BC
:106330004B015C012C853D854E855F85821A930A51
:10634000A40AB50AB7FE08C0B094A09490948094B3
:10635000811C911CA11CB11C092C000CAA08BB08B3
:106360002114310419F580EF94E00E94391682E17E
:1063700094E00E9439168FE893E00E9439168A89CA
:106380009B890E94341682E194E00E9439168FE0C6
:1063900098E00E943916C501B4010E94B95442E048
:1063A0000E94511A0E945D140E943A1685E090E006
:1063B000EE81FF819183808345E050E0B60188A1A2
:1063C00099A129DCC6010E94BB0C0E94E6140E9420
:1063D000D019288539852130310509F4BAC0223019
:1063E000310509F4C1C00E945D1480922E0990927B
:1063F0002F09A0923009B09231090E945D140E94C9
:10640000261BEE81FF811182108250E040E0B60130
:1064100088A199A100DC70E060E0C6010E945116DD
:106420000E945D1430925E0820925D08BACCC601CD
:106430000E948F0CF8011082F2CE81ED9CE00E9448
:10644000D5078F7D8534910509F03ECF84EB94E02C
:106450000E9439160E945D1421E0FC01268786E522
:1064600092E00E9439160E945D140E943A1622247E
:106470002394312C11E029CF11113ACFE889F98901
:1064800060817181072E000C880B990B0E94B95412
:106490009B01AC01EB81FC816081718182819381E0
:1064A0000E94B35487FF24CFC6010E94770D82015A
:1064B0000F5F1F4FF501208131814281538160E5DB
:1064C00073EC80E090E00E94E555C9010E94030A48
:1064D000FFEF4F1A5F0A6F0A7F0AF50120813181B1
:1064E00042815381A3E0B0E00E9401569B01AC01C0
:1064F000C301B2010E94E555672B682B692BB9F4E3
:1065000082E592E00E9439160E945D140E943A16BC
:1065100081E993E00E94391688E095E00E943916DF
:10652000C8010E9434168EED97E00E943916C6010C
:106530000E94580CF501208131814281538160E530
:1065400073EC80E090E00E94E555C9010E94030AC7
:10655000A2CE0E945D148092320990923309A092DB
:106560003409B092350949CF0E945D1480923609F2
:1065700090923709A0923809B09239093ECF0E9413
:10658000710CB3CEFA01DB01A359BF4F2C9122232A
:1065900031F122E030E0DB01A159BF4F4C9144239F
:1065A00011F023E030E0DB01A259BF4F4C914423AE
:1065B00011F024E030E0DB01A059BF4F4C9144239F
:1065C00011F026E030E0408151814217530761F01D
:1065D000121613063CF431832083A9011CCB30E052
:1065E00020E0D9CF1182108208952F923F924F92CE
:1065F0005F926F927F928F929F92AF92BF92CF9253
:10660000DF92EF92FF920F931F93CF93DF93CDB75B
:10661000DEB7EC970FB6F894DEBF0FBECDBF1C01FE
:106620002A013B010B871C872D873E8764960EADA0
:106630001FAD6497FC01EB54FD4F60817181828135
:1066400093810E94B954A30192010E9418550E949F
:106650000F576B8F7C8F8D8F9E8FF101E754FD4F0D
:1066600060817181828193810E94B9542B853C8520
:106670004D855E850E9418550E940F576BA37CA321
:106680008DA39EA3F101E354FD4F6081718182814E
:1066900093810E94B954A70196010E9418550E9447
:1066A0000F576BA77CA78DA79EA70E94640A6B87D4
:1066B0007C878D879E87F101EA5CFD4F11821082F5
:1066C0003296118210823E96A114B10461F0C50188
:1066D000B0E0A0E040815181628173818417950709
:1066E000A607B70714F0A080B180F101E65BFD4F6B
:1066F00080819181A281B3818114910441F0A40130
:1067000070E060E0481759076A077B070CF04C01FE
:10671000F101E25BFD4F80819181A281B38101157E
:10672000110541F0A80170E060E0481759076A07B9
:106730007B070CF08C01210120E1420E511CC501A8
:10674000B0E0A0E0F10186A797A7A0ABB1AB310103
:10675000F4E96F0E711CB12CA12CD3015E968D92C1
:106760009D92AD92BC9291974101B8EE8B1ABEEF0B
:106770009B0A30E020E0F401068F178F20A331A39D
:106780000E945D140E945D140E945D140E945D14BD
:1067900020912E0930912F094091300950913109F3
:1067A0002B8B3C8B4D8B5E8B0E945D14809132094C
:1067B00090913309A0913409B09135098F87988B56
:1067C000A98BBA8B0E945D14A0903609B09037094E
:1067D000C0903809D0903909F101EF53FD4F108274
:1067E00011821282138234961082118212821382D5
:1067F0003496108211821282138234961182108292
:1068000032961182108232961182108232962B8932
:106810003C894D895E89208331834283538334963A
:106820008F859889A989BA8980839183A283B3834C
:106830003496A082B182C282D3826596EFAC65970E
:106840000B8D1C8D2D8D3E8D4B895C896D897E89CC
:10685000C2010E94E00C8823F9F08EE492E00E94CD
:10686000391685E394E00E943916F101E85AFF4F8A
:106870006081718182819381E35AFD4F2081318152
:10688000428153810E94E555CA01B9010E940C164C
:106890000E945D140E943A166696EFAC66970BA1B3
:1068A0001CA12DA13EA14F85588969897A89C30110
:1068B0000E94E00C8823F9F08AE492E00E943916E5
:1068C00085E494E00E943916F101E452FF4F6081A3
:1068D000718182819381E352FE4F20813181428117
:1068E00053810E94E555CA01B9010E940C160E940D
:1068F0005D140E943A166796EFAC67970BA51CA52E
:106900002DA53EA5B601A501C4010E94E00C882377
:10691000F9F086E492E00E94391685E594E00E9441
:106920003916F101E05AFE4F6081718182819381B5
:10693000E35AFE4F20813181428153810E94E55507
:10694000CA01B9010E940C160E945D140E943A16F9
:10695000D10155961C92F101E756FF4F1082EC577A
:10696000FF4F10820E94E6140E94D019C2010E94BB
:10697000910EC3010E94910EC4010E94910EF1017B
:10698000E35CFD4FFCA7EBA781E090E0918380835F
:106990007101F1ECEF1AFDEFFF0AD7018D939C9383
:1069A00081010F5B1D4FF8019183808341E050E02E
:1069B000B201C10130D9D7014D915C91B301C10140
:1069C0002AD9F80140815181B401C10124D911E0D3
:1069D000F101EE5DFC4F1083C2010E94CD0CC3019A
:1069E0000E94CD0CC4010E94CD0C64E670E080E0F2
:1069F00090E00E94330AC101865C9D4FDC011C932C
:106A000011961C93A101445C5D4FFA0110836596B9
:106A1000FFAD6597F1110FC066962FAD66972111F6
:106A200005C067963FAD6797332339F19101275829
:106A30003F4FF90110826696FFAD6697F11105C0D0
:106A4000910123503F4FF90110826796FFAD679780
:106A5000F11105C091012F573E4FF9011082659643
:106A60002FAD6597FC01208366963FAD66973C93FA
:106A70006796EFAD6797DA01EC93C2010E94201789
:106A8000C3010E942017C4010E942017C2010E9466
:106A9000D60DC3010E94D60DC4010E94D60D0E94DE
:106AA0005D14DC011E968C918F87B12CA12CF10115
:106AB000E65CFD4FFC8BEB8B9101255C3D4F3C8FE1
:106AC0002B8FA101445C5D4F5CA34BA3C101835C90
:106AD0009D4F9AAB89ABD101A15CBD4FBCABABABB9
:106AE0003796FEABEDAB2F5B314038AB2FA74F5342
:106AF0005F4F58AF4FAB8C549F4F9AAF89AFAC5696
:106B0000BF4FBCAFABAFEB89FC89808181110AC05C
:106B1000AB8DBC8D8C91811105C0EBA1FCA1808156
:106B2000882319F0FF85FF2369F08101005D1D4F67
:106B3000F80180819181892B09F47AC4C1010E94F6
:106B4000F72CF6CF49A95AA9B201C1011BDD4BA907
:106B50005CA9B301C10116DD4DA95EA9B401C10153
:106B600011DDC2010E943E0EC3010E943E0EC4010F
:106B70000E943E0EAFA5B8A98C918823A9F0C2014E
:106B80000E942017EFA8F8AC09AD1AAD2BAD3CADB3
:106B9000A1014F535D4FB10164567E4FC2010E9467
:106BA000EE10EFA5F8A910826101D394D6018C9163
:106BB0008823C9F0C3010E9420177101B2E0EB1ACB
:106BC000BDEFFB0A81010B501D4F910129523D4F32
:106BD000A1014B535D4FB10164537E4FC3010E942D
:106BE000EE10F60110826101FCE7CF1AFEEFDF0A1A
:106BF000D6018C918823C9F0C4010E94201771012D
:106C0000B1E0EB1ABDEFFB0A810107501D4F910166
:106C100025523D4FA10147535D4FB10164507E4F56
:106C2000C4010E94EE10F6011082810107581F4F27
:106C3000D8018C918823C1F1F101E551FD4F6081AC
:106C40007181072E000C880B990B0E94B9549B018F
:106C5000AC01F101EF53FD4F60817181828193811D
:106C60000E944057181604F5F801108261E973E09C
:106C70000D541E4FC8010E94B52D64E275E0C80195
:106C80000E94B52D6EED77E0C8010E94B52D659686
:106C9000FFAD6597FF2309F434C1F101EC5AFF4FB2
:106CA0001082118212821382810103501F4FD8017A
:106CB0008C918823C1F1F101E351FD4F6081718115
:106CC000072E000C880B990B0E94B9549B01AC0154
:106CD000F101EB53FD4F60817181828193810E94AC
:106CE0004057181604F5F801108261E973E0015D60
:106CF0001E4FC8010E94B52D6CE475E0C8010E94CA
:106D0000B52D6EED77E0C8010E94B52D6696FFADFA
:106D10006697FF2309F4F9C0F101E852FF4F108292
:106D200011821282138281010F571E4FD8018C915C
:106D30008823C1F1F101E151FD4F60817181072E7E
:106D4000000C880B990B0E94B9549B01AC01F10116
:106D5000E753FD4F60817181828193810E9440578A
:106D6000181604F5F801108261E973E005551F4F0C
:106D7000C8010E94B52D64E775E0C8010E94B52DD9
:106D80006EED77E0C8010E94B52D6796FFAD67975D
:106D9000FF2309F4BEC0F101E45AFE4F10821182B4
:106DA0001282138260E0C2010E945B0D882339F0D9
:106DB000F101EC5AFF4F108211821282138260E0BF
:106DC000C3010E945B0D882339F0F101E852FF4FA7
:106DD000108211821282138260E0C4010E945B0D56
:106DE000882339F0F101E45AFE4F10821182128299
:106DF0001382F101E758FF4F8081AB89BC898C93E6
:106E0000EC57FF4F8081EB8DFC8D8083F101EF57B4
:106E1000FE4F8081ABA1BCA18C93ED52F14020814B
:106E20003181428153812FA338A749A75AA7EC5734
:106E3000FF4F80819181A281B3818F839887A98739
:106E4000BA87EC57FF4FC080D180E280F3800E9468
:106E50005D142FA138A549A55AA520932E0930937A
:106E60002F0940933009509331090E945D148F819E
:106E70009885A985BA858093320990933309A093A8
:106E80003409B09335090E945D14C0923609D0923E
:106E90003709E0923809F09239090E94E614AB896B
:106EA000BC898C91882309F46AC00E94640A2B85EE
:106EB0003C854D855E85621773078407950768F5E5
:106EC0000E94640A2B853C854D855E856217730799
:106ED0008407950708F053C00E94640A6B017C0187
:106EE000F101E755FD4F2081318142815381A8EEA8
:106EF000B3E00E9401566C157D058E059F0550F18B
:106F00003EC073E0A72EB12CCFCE63E0A62EB12CED
:106F10000ACF53E0A52EB12C45CF0E94640A6B0125
:106F20007C012B853C854D855E85C21AD30AE40A17
:106F3000F50AF101E755FD4F2081318142815381EE
:106F4000A8EEB3E00E9401566C157D058E059F05E5
:106F500008F0B6CF62E472E08101045D1D4FC80104
:106F60000E94B52D6EED77E0C8010E94B52D6CE949
:106F700075E0C8010E94B52D42E0A42EB12CAB8D66
:106F8000BC8D8C91882309F45DC00E94640A2B8516
:106F90003C854D855E85621773078407950708F564
:106FA0000E94640A2B853C854D855E8562177307B8
:106FB0008407950708F046C00E94640A6B017C01B3
:106FC000F101E355FD4F2081318142815381A8EECB
:106FD000B3E00E9401566C157D058E059F05E8F013
:106FE00031C00E94640A6B017C012B853C854D8574
:106FF0005E85C21AD30AE40AF50AF101E355FD4F92
:107000002081318142815381A8EEB3E00E94015674
:107010006C157D058E059F0518F66EE372E0810103
:10702000045D1D4FC8010E94B52D6EED77E0C801CB
:107030000E94B52D61EB75E0C8010E94B52D32E0CC
:10704000A32EB12CABA1BCA18C91882309F45DC007
:107050000E94640A2B853C854D855E856217730707
:107060008407950708F50E94640A2B853C854D85A9
:107070005E85621773078407950708F046C00E9473
:10708000640A6B017C01F101EF54FD4F20813181D5
:1070900042815381A8EEB3E00E9401566C157D0534
:1070A0008E059F05E8F031C00E94640A6B017C01E7
:1070B0002B853C854D855E85C21AD30AE40AF50A04
:1070C000F101EF54FD4F2081318142815381A8EEBF
:1070D000B3E00E9401566C157D058E059F0518F6DC
:1070E0006AE372E08101045D1D4FC8010E94B52D65
:1070F0006EED77E0C8010E94B52D66EC75E0C80121
:107100000E94B52D22E0A22EB12C81ED9CE00E94C0
:10711000F707181619060CF040C081ED9CE00E949C
:10712000D5078F7D85349105C1F564EB74E0C1010D
:10713000845D9D4F0E94B52D86E592E00E94391630
:107140000E945D140E943A16F101E758FF4F108229
:10715000EC57FF4F1082EC57FF4F1082AB89BC8970
:107160001C92EB8DFC8D1082ABA1BCA11C92B1E0F6
:10717000BF87AA24A394B12C6BED75E0C101845D97
:107180009D4F0E94B52DEB89FC891082AB8DBC8D83
:107190001C92EBA1FCA1108203C0A114B10461F701
:1071A000C1010E94F72CF101E85CFD4F80819181C3
:1071B0000196918380838D3291400CF4A4CCD1014F
:1071C000A05DBD4F8D919C911197892B09F09BCCAF
:1071D00014968D919C91892B09F095CC1182108287
:1071E0003297808191818130910581F182309105C2
:1071F00009F4F4C0892BC1F462E572E08101045DF9
:107200001D4FC8010E94B52D0E945D14CE0101964C
:107210000E94BE2DBE016F5F7F4FC8010E94052EE8
:10722000CE0101960E94B129F101EA5CFD4F8081F7
:1072300091810196833091050CF0F7C09183808392
:10724000F101EC5CFD4F118210825DCC0E945D1457
:107250008C01FC0180819181A281B38118161906ED
:107260001A061B0644F081E090E0A0E0B0E08083C5
:107270009183A283B383F80184819581A681B7812C
:10728000181619061A061B0644F081E090E0A0E0EB
:10729000B0E084839583A683B783F80180859185C8
:1072A000A285B385181619061A061B0644F081E05C
:1072B00090E0A0E0B0E080879187A287B3871A8230
:1072C00019821C821B821E821D82CE0101960E94A1
:1072D000342A60E274E0CE0101960E94B52D65E388
:1072E00074E0CE0101960E94B52D60912E09709137
:1072F0002F0980913009909131090E94B9546B0196
:107300007C01D8016D917D918D919C910E94B95421
:107310009B01AC01C701B6010E94A756AB01BC019D
:10732000CE0101960E94592D65E474E0CE010196CC
:107330000E94B52D60913209709133098091340912
:10734000909135090E94B9546B017C01F801648168
:107350007581868197810E94B9549B01AC01C70158
:10736000B6010E94A756AB01BC01CE0101960E9456
:10737000592D65E574E0CE0101960E94B52D60910E
:1073800036097091370980913809909139090E9426
:10739000B9546B017C01D80118966D917D918D9146
:1073A0009C911B970E94B9549B01AC01C701B60187
:1073B0000E94A756AB01BC01CE0101960E94592D37
:1073C000BE016F5F7F4F8101045D1D4FC8010E94A8
:1073D000052ECE0101960E94B12916CF67EE75E009
:1073E0008101045D1D4FC8010E94B52D65E374E065
:1073F000C8010E94B52D70E060E0C8010E94892D8F
:1074000065E474E0C8010E94B52D70E060E0C80139
:107410000E94892D65E574E0C8010E94B52D70E0D9
:1074200060E0C8010E94892DEFCE1182108208CF42
:107430008BEE95E00E9439166596FFAD6597FF23A8
:1074400079F1A114B104B9F52F85211134C086E377
:1074500092E00E9439160E945D140E943A166696C8
:107460003FAD6697332341F082E392E00E943916E4
:107470000E945D140E943A1667968FAD6797882325
:10748000D1F0A114B104B9F49F85911114C08EE21A
:1074900092E00E9439160E945D140E943A160BC0B9
:1074A00066965FAD6697552339F3A114B10419F4BC
:1074B0004F854423C9F285E090E0ABA5BCA58D9330
:1074C0009C938101015C1D4FF801918380839101A0
:1074D0002F5B3D4F3C872B87D9018D939C9345E0D3
:1074E00050E0B201C1010E940B2EF8014081518190
:1074F000B301C1010E940B2EAB85BC854D915C91FF
:10750000B401C1010E940B2EC1010E942D14F10192
:10751000EC5AFF4F20813181428153812F8F38A354
:1075200049A35AA3EC57FF4F80819181A281B38177
:107530008F8B988FA98FBA8FEC57FF4FC080D18067
:10754000E280F3800E945D142F8D38A149A15AA1D9
:1075500020932E0930932F0940933009509331091D
:107560000E945D148F89988DA98DBA8D8093320900
:1075700090933309A0933409B09335090E945D14A8
:10758000C0923609D0923709E0923809F092390951
:107590000E94E6140E94D0190E945D140E94261BCE
:1075A000C1010E94C61BABA5BCA51D921C92F8018F
:1075B00011821082AB85BC851D921C9250E040E088
:1075C000B201C1010E940B2EF80140815181B3012B
:1075D000C1010E940B2EAB85BC854D915C91B4011D
:1075E000C1010E940B2EC1010E942D14BF85BB2337
:1075F00041F00E945D1421E0FC012687AA24A39497
:10760000B12C89EF95E00E943916C5010E9434160D
:107610008EED97E00E9439160E945D14B0925E08CC
:10762000A0925D08C501EC960FB6F894DEBF0FBEC0
:10763000CDBFDF91CF911F910F91FF90EF90DF9021
:10764000CF90BF90AF909F908F907F906F905F9002
:107650004F903F902F9008958F929F92AF92BF923C
:10766000CF92DF92EF92FF920F931F930E946D2CA7
:1076700062E070E00E94592E892BD1F40E946D2C9B
:1076800021E02F931F921F921F921F92912C812C09
:10769000B12CA12CC12CD12C760197018601B70108
:1076A000A6010E94F5320F900F900F900F900F904F
:1076B00090E080E01F910F91FF90EF90DF90CF90CE
:1076C000BF90AF909F908F9008952F923F924F92CE
:1076D0005F926F927F928F929F92AF92BF92CF9262
:1076E000DF92EF92FF920F931F93CF93DF930E944D
:1076F0003B1D8091150A9091160A019709F055C01B
:1077000086EF9FEFD0E0C0E02C01990F6608770864
:10771000C330D10509F44CC0C530D10509F448C0C7
:10772000C130D10509F444C00E946D2C1F9221E0A4
:107730002F931F921F921F92912C812CB12CA12C60
:10774000C12CD12C760197018601B701A6010E94B8
:10775000F5320F900F900F900F900F900E945D14D4
:1077600020905D0830905E080E945D14FC018685C3
:10777000811106C0232821F42196C730D10541F696
:1077800090E080E0DF91CF911F910F91FF90EF90FB
:10779000DF90CF90BF90AF909F908F907F906F9031
:1077A0005F904F903F902F9008958AE090E0AACF8D
:1077B0000E946D2C1C01C301B2010E94B9548B01BF
:1077C0009C011F921F921F921F921F92912C812C3D
:1077D000B12CA12CC12CD12C7601B701A601C1017D
:1077E000B6CF4F925F926F927F928F929F92AF929D
:1077F000BF92CF92DF92EF92FF920F931F93CF939E
:10780000DF9300D01F92CDB7DEB70E943B1D4090A2
:10781000250A5090260A6090270A7090280A0E9434
:107820003B1D8090290A90902A0AA0902B0AB090C4
:107830002C0A0E945D14C0902E09D0902F09E09070
:107840003009F09031090E945D14C701B6010E9411
:10785000B9546B017C01C301B2010E94B9549B0170
:10786000AC01C701B6010E94A7562B013C016091F3
:1078700032097091330980913409909135090E9441
:10788000B9546B017C01C501B4010E94B9549B013C
:10789000AC01C701B6010E94A75669837A838B8326
:1078A0009C830E946D2C1F921F921F921F921F9209
:1078B000912C812CB12CA12CC12CD12C76010981C9
:1078C0001A812B813C81B301A2010E94F5320E94F2
:1078D0006D2C1F921F921F921F921F92970186017B
:1078E000B301A2010E94F5320E946D2C1F921F92DB
:1078F0001F921F921F929701B701A6010E94F532B5
:107900000FB6F894DEBF0FBECDBF90E080E00F90C1
:107910000F900F900F90DF91CF911F910F91FF90DB
:10792000EF90DF90CF90BF90AF909F908F907F901F
:107930006F905F904F9008952F923F924F925F9279
:107940006F927F928F929F92AF92BF92CF92DF926F
:10795000EF92FF920F931F93CF93DF930E943B1DF3
:107960008091150A9091160A019709F055C086EF8B
:107970009FEFD0E0C0E02C01990F66087708C33074
:10798000D10509F44CC0C530D10509F448C0C13057
:10799000D10509F444C00E946D2C1F921F9221E072
:1079A0002F931F921F92912C812CB12CA12CC12CB2
:1079B000D12C760197018601B701A6010E94F5320C
:1079C0000F900F900F900F900F900E945D142090D9
:1079D0005D0830905E080E945D14FC01868581116F
:1079E00006C0232821F42196C730D10541F690E046
:1079F00080E0DF91CF911F910F91FF90EF90DF908A
:107A0000CF90BF90AF909F908F907F906F905F903E
:107A10004F903F902F9008958AE090E0AACF0E9467
:107A20006D2C1C01C301B2010E94B954AB01BC0111
:107A30001F921F921F921F921F92912C812CB12C8A
:107A4000A12CC12CD12C760197018601C101B6CFA2
:107A50008F929F92AF92BF92CF92DF92EF92FF925E
:107A60000F931F93CF93DF93EB010E946D2C8A88B5
:107A70009B88AE84BF84CA84DB84EC84FD840E8141
:107A80001F81288539854A815B816C817D811F92A8
:107A90001F921F92EF89EF93EE89EF930E94F532C8
:107AA0000F900F900F900F900F9090E080E0DF917B
:107AB000CF911F910F91FF90EF90DF90CF90BF90EB
:107AC000AF909F908F9008952F923F924F925F9228
:107AD0006F927F928F929F92AF92BF92CF92DF92DE
:107AE000EF92FF920F931F93CF93DF930E946D2C21
:107AF00021E02F931F921F921F921F92912C812C95
:107B0000B12CA12CC12CD12C760197018601B70193
:107B1000A6010E94F5320E943B1D0F900F900F901E
:107B20000F900F908091150A9091160A019709F015
:107B300055C086EF9FEFD0E0C0E02C01990F66089A
:107B40007708C330D10509F44CC0C530D10509F41C
:107B500048C0C130D10509F444C00E946D2C21E019
:107B60002F931F921F921F921F92912C812CB12C48
:107B7000A12CC12CD12C760197018601B701A60159
:107B80000E94F5320F900F900F900F900F900E946F
:107B90005D1420905D0830905E080E945D14FC0129
:107BA0008685811106C0232821F42196C730D1058E
:107BB00041F690E080E0DF91CF911F910F91FF900F
:107BC000EF90DF90CF90BF90AF909F908F907F907D
:107BD0006F905F904F903F902F9008958AE090E0D3
:107BE000AACF0E946D2C1C01C301B2010E94B9549E
:107BF0006B017C011F921F921F921F921F92912C6A
:107C0000812CB12CA12C00E010E09801B901A80151
:107C1000C101B6CF8F929F92AF92BF92CF92DF9267
:107C2000EF92FF920F931F930E946D2C70E060E023
:107C30000E94592E892BD1F40E946D2C1F921F9205
:107C400021E02F931F921F92912C812CB12CA12CFB
:107C5000C12CD12C760197018601B701A6010E94A3
:107C6000F5320F900F900F900F900F9090E080E002
:107C70001F910F91FF90EF90DF90CF90BF90AF904A
:107C80009F908F9008958F929F92AF92BF92CF92C4
:107C9000DF92EF92FF920F931F930E946D2C61E091
:107CA00070E00E94592E892BD1F40E946D2C1F92F6
:107CB00021E02F931F921F921F92912C812CB12CA7
:107CC000A12CC12CD12C760197018601B701A60108
:107CD0000E94F5320F900F900F900F900F9090E050
:107CE00080E01F910F91FF90EF90DF90CF90BF90B9
:107CF000AF909F908F9008951F920F920FB60F92A2
:107D000011240BB60F922F933F934F935F936F9372
:107D10007F938F939F93AF93BF93EF93FF9381EDE7
:107D20009CE00E940C08FF91EF91BF91AF919F9151
:107D30008F917F916F915F914F913F912F910F9014
:107D40000BBE0F900FBE0F901F9018951F920F92B1
:107D50000FB60F9211240BB60F922F938F939F9310
:107D6000EF93FF93E091E10CF091E20C8081E091C0
:107D7000E70CF091E80C82FD1DC090818091EA0C27
:107D80008F5F8F732091EB0C821741F0E091EA0C2A
:107D9000F0E0EF52F34F958F8093EA0CFF91EF9153
:107DA0009F918F912F910F900BBE0F900FBE0F9050
:107DB0001F9018958081F2CF1F920F920FB60F92ED
:107DC00011242F933F938F939F93AF93BF938091F1
:107DD000240890912508A0912608B0912708309199
:107DE000230823E0230F2D3758F50196A11DB11D5F
:107DF000209323088093240890932508A0932608B5
:107E0000B09327088091280890912908A0912A080A
:107E1000B0912B080196A11DB11D80932808909365
:107E20002908A0932A08B0932B08BF91AF919F9186
:107E30008F913F912F910F900FBE0F901F9018952B
:107E400026E8230F0296A11DB11DD2CF1F920F92DB
:107E50000FB60F9211240BB60F922F933F934F93AF
:107E60005F936F937F938F939F93AF93BF93EF93A2
:107E7000FF9348E251E064E271E090E080E00E940C
:107E8000730BFF91EF91BF91AF919F918F917F9174
:107E90006F915F914F913F912F910F900BBE0F907B
:107EA0000FBE0F901F9018951F920F920FB60F9252
:107EB00011240BB60F922F933F934F935F936F93C1
:107EC0007F938F939F93AF93BF93EF93FF9348EA72
:107ED00050E064EA70E083E090E00E94730BFF9151
:107EE000EF91BF91AF919F918F917F916F915F9132
:107EF0004F913F912F910F900BBE0F900FBE0F909F
:107F00001F9018951F920F920FB60F9211240BB667
:107F10000F922F933F934F935F936F937F938F9322
:107F20009F93AF93BF93EF93FF9348E950E064E9C9
:107F300070E082E090E00E94730BFF91EF91BF919F
:107F4000AF919F918F917F916F915F914F913F91F1
:107F50002F910F900BBE0F900FBE0F901F90189592
:107F60001F920F920FB60F9211240BB60F922F9300
:107F70003F934F935F936F937F938F939F93AF93B1
:107F8000BF93EF93FF9348E850E064E870E081E02E
:107F900090E00E94730BFF91EF91BF91AF919F9181
:107FA0008F917F916F915F914F913F912F910F90A2
:107FB0000BBE0F900FBE0F901F9018951F920F923F
:107FC0000FB60F9211240BB60F922F933F934F933E
:107FD0005F936F937F938F939F93AF93BF93EF9331
:107FE000FF93E0912D08F0912E081995FF91EF91E4
:107FF000BF91AF919F918F917F916F915F914F91C1
:108000003F912F910F900BBE0F900FBE0F901F90BE
:108010001895FF920F931F93CF93DF93EC01F62EE9
:108020008C01065F1F4F1B861A861D861C861F86C5
:108030001E86C8010E94342AF886198670E060E026
:10804000C801DF91CF911F910F91FF900C940F2ADF
:108050001092D40C1092D30C88EE93E0A0E0B0E024
:108060008093D50C9093D60CA093D70CB093D80CDA
:1080700082E793E09093D20C8093D10C85EC90E052
:108080009093DE0C8093DD0C84EC90E09093E00CF8
:108090008093DF0C80EC90E09093E20C8093E10CF5
:1080A00081EC90E09093E40C8093E30C82EC90E000
:1080B0009093E60C8093E50C86EC90E09093E80CAE
:1080C0008093E70C1092EA0C1092EB0C1092EC0CDF
:1080D0001092ED0C68E18DEC93E19BDF6CE18DED8E
:1080E00093E197DF67E18DEE93E193DF6DE18DEF33
:1080F00093E18FDF68E18DE893E18BDF6CE18DE93F
:1081000093E187DF67E18DEA93E183DF6DE18DEB3A
:1081100093E17FDF68E18DE493E17BDF6CE18DE546
:1081200093E177DF67E18DE693E173DF6DE18DE742
:1081300093E16FDF68E18DE093E16BDF6CE18DE14E
:1081400093E167DF67E18DE293E163DF6DE18DE34A
:1081500093E15FDF68E18DEC92E15BDF6CE18DED37
:1081600092E157DF67E18DEE92E153DF6DE18DEF34
:1081700092E14FDF68E18DE892E14BDF6CE18DE940
:1081800092E147DF67E18DEA92E143DF6DE18DEB3C
:1081900092E13FDF68E18DE492E13BDF6CE18DE548
:1081A00092E137DF67E18DE692E133DF6DE18DE744
:1081B00092E12FDF68E18DE092E12BDF6CE18DE150
:1081C00092E127DF67E18DE292E123DF6DE18DE34C
:1081D00092E11FDF68E18DEC91E11BDF6CE18DED39
:1081E00091E117DF67E18DEE91E113DF6DE18DEF36
:1081F00091E10FDF68E18DE891E10BDF6CE18DE942
:1082000091E107DF67E18DEA91E103DF6DE18DEB3D
:1082100091E1FFDE68E18DE491E1FBDE6CE18DE54B
:1082200091E1F7DE67E18DE691E1F3DE6DE18DE747
:1082300091E1EFDE68E18DE091E1EBDE6CE18DE153
:1082400091E1E7DE67E18DE291E1E3DE6DE18DE34F
:1082500091E1DFDEEFEFFDE02FEF48EB5BE0809197
:10826000FE0D803308F0E3C091E0980F9093FE0D6F
:10827000808390E0DC01AA0FBB1FA80FB91FA25991
:10828000B24F12965C934E93119733968EE0EB307B
:10829000F80729F768E18DEC90E1BBDE6CE18DED2C
:1082A00090E1B7DE67E18DEE90E1B3DE6DE18DEF39
:1082B00090E1AFDE82E090E00E943A4F24E833E0A4
:1082C000FC013183208390930C0E80930B0E68E1A8
:1082D0008DE890E19EDE6CE18DE990E19ADE67E148
:1082E0008DEA90E196DE6DE18DEB90E192DE68E142
:1082F0008DE490E18EDE6CE18DE590E18ADE67E150
:108300008DE690E186DE6DE18DE790E182DE68E149
:108310008DE090E17EDE6CE18DE190E17ADE67E157
:108320008DE290E176DE6DE18DE390E172DE68E151
:108330008DEC9FE06EDE6CE18DED9FE06ADE67E123
:108340008DEE9FE066DE6DE18DEF9FE062DE68E11D
:108350008DE89FE05EDE6CE18DE99FE05ADE67E12B
:108360008DEA9FE056DE6DE18DEB9FE052DE68E125
:108370008DE49FE04EDE6CE18DE59FE04ADE67E133
:108380008DE69FE046DE6DE18DE79FE042DE68E12D
:108390008DE09FE03EDE6CE18DE19FE03ADE67E13B
:1083A0008DE29FE036DE6DE18DE39FE032DE68E135
:1083B0008DEC9EE02EDE6CE18DED9EE02ADE67E125
:1083C0008DEE9EE026DE6DE18DEF9EE022DE68E11F
:1083D0008DE89EE01EDE6CE18DE99EE01ADE67E12D
:1083E0008DEA9EE016DE6DE18DEB9EE012DE68E127
:1083F0008DE49EE00EDE6CE18DE59EE00ADE67E135
:108400008DE69EE006DE6DE18DE79EE002DE68E12E
:108410008DE09EE0FEDD6CE18DE19EE0FADD67E13E
:108420008DE29EE0F6DD6DE18DE39EE0F2CD2083EE
:108430002CCF789484B5826084BD84B5816084BD7E
:1084400085B5826085BD85B5816085BD80916E00F2
:10845000816080936E001092810080918100826023
:108460008093810080918100816080938100809160
:1084700080008160809380008091B100846080934F
:10848000B1008091B00081608093B0008091910034
:10849000826080939100809191008160809391002F
:1084A000809190008160809390008091A100826013
:1084B0008093A1008091A10081608093A1008091B0
:1084C000A00081608093A000809121018260809350
:1084D00021018091210181608093210180912001FF
:1084E00081608093200180917A00846080937A007B
:1084F00080917A00826080937A0080917A00816016
:1085000080937A0080917A00806880937A0010923C
:10851000C100E091E10CF091E20C82E08083E091F7
:10852000DD0CF091DE0C1082E091DF0CF091E00C9C
:1085300010E110831092E90CE091E50CF091E60C4B
:1085400086E08083E091E30CF091E40C808180610F
:108550008083E091E30CF091E40C8081886080835B
:10856000E091E30CF091E40C808180688083E091DD
:10857000E30CF091E40C80818F7D808364E670E0F1
:1085800080E090E00E94330A8FE592E00E94391665
:108590008DE592E00E94391684E096E00E9439163B
:1085A0008AE592E00E9439168FE592E00E94391622
:1085B0008DE592E00E9439168EE196E00E94391610
:1085C0008AE592E00E94391661E089E10E948909FA
:1085D00061E08BE10E94890961E08AE10E948909DA
:1085E00062E085E40E94890962E084E40E948909CE
:1085F00061E089E10E945C0960E08BE10E945C0916
:1086000060E08AE10E945C0961E08FE10E948909D3
:1086100061E081E20E94890961E080E20E948909AB
:1086200062E083E40E94890962E082E40E94890991
:1086300061E08FE10E945C0960E081E20E945C09D8
:1086400060E080E20E945C0961E082E20E948909A8
:1086500061E084E20E94890961E083E20E94890965
:1086600062E081E40E94890962E080E40E94890955
:1086700061E082E20E945C0960E084E20E945C09A1
:1086800060E083E20E945C0961E08EE00E9489095B
:1086900061E08EE10E94890961E08FE00E94890912
:1086A00061E08EE00E945C0960E08EE10E945C095E
:1086B00060E08FE00E945C0961E088E20E94890925
:1086C00061E089E20E94890961E085E20E948909EE
:1086D00060E088E20E945C0960E089E20E945C0937
:1086E00060E085E20E945C0961E08DE00E948909FA
:1086F00061E089E00E94890961E088E00E948909BF
:1087000061E087E00E94890961E08AE00E948909AE
:1087100061E08CE00E94890960E08DE00E945C09C4
:1087200060E089E00E945C0960E088E00E945C09EA
:1087300060E087E00E945C0960E08AE00E945C09DA
:1087400060E08CE00E945C0962E08FE30E9489098E
:1087500062E08BE30E94890961E084E00E9489095C
:1087600061E085E00E94890961E086E00E94890954
:1087700061E087E00E94890960E084E00E945C0972
:1087800060E085E00E945C0960E086E00E945C0990
:1087900060E087E00E945C098FE592E00E94391654
:1087A0008DE592E00E9439168FE396E00E9439161B
:1087B0008AE592E00E9439160E943B1D0E942E1A03
:1087C0008FE592E00E9439168DE592E00E943916FD
:1087D0008FE496E00E9439168AE592E00E943916ED
:1087E0008FE592E00E9439168DE592E00E943916DD
:1087F00080E696E00E9439168AE592E00E943916DA
:108800000E946D2CEC0140960E947111CE018C5695
:108810009F4F0E947111CE01885E9E4F0E94711180
:108820008FE592E00E9439168DE592E00E9439169C
:1088300085E796E00E9439168AE592E00E94391693
:108840000E946D2C0E94C7288FE592E00E94391685
:108850008DE592E00E9439168DE896E00E94391667
:108860008AE592E00E9439160E946D2C0E948127B1
:108870008FE592E00E9439168DE592E00E9439164C
:1088800084EA96E00E9439168AE592E00E94391641
:1088900061E089E10E945C0961E08EE00E945C0970
:1088A00061E08FE10E945C0961E082E20E945C0964
:1088B0008FE592E00E9439168DE592E00E9439160C
:1088C0008AEB96E00E9439168AE592E00E943916FA
:1088D0000E94341E0E94041E0E94640A0E94640AC0
:1088E00060932F087093300880933108909332087A
:1088F0008FE592E00E9439168DE592E00E943916CC
:108900008AEC96E00E9439168AE592E00E943916B8
:108910000E94EE1464E070E08FEF9DE00E94EC0A8C
:1089200065E070E082E09EE00E94EC0A66E070E0A4
:1089300085E09EE00E94EC0A67E070E088E09EE03F
:108940000E94EC0A8FE592E00E9439168DE592E0D4
:108950000E94391686ED96E00E9439168AE592E06B
:108960000E94391686E89CE290932E0880932D0889
:10897000C1E0C0936F001093810010928000C093FB
:108980002C0880E092E0909387008093860081E13C
:1089900080938100109281001092850010928400D3
:1089A00080912C088061809381000E94640A60930A
:1089B0003E0970933F0980934009909341098FE5E8
:1089C00092E00E9439168DE592E00E94391686EEFB
:1089D00096E00E9439168AE592E00E9439160E94BC
:1089E0003B1D8091510990915209A0915309B0917A
:1089F00054090197A105B10559F50E943B1D8091CD
:108A0000990990919A09A0919B09B0919C090197AD
:108A1000A105B105E9F48BEF96E00E9439160E949A
:108A20006D2CCF931F921F921F921F92912C812C1D
:108A3000B12CA12CC12CD12C760197018601B70154
:108A4000A6010E94F5320F900F900F900F900F909B
:108A50000E943B1D8091510990915209A0915309A8
:108A6000B09154090197A105B10561F50E943B1D24
:108A70008091950990919609A0919709B0919809D4
:108A80000197A105B105F1F483E197E00E94391641
:108A90000E946D2C1F9221E02F931F921F921F9214
:108AA000912C812CB12CA12CC12CD12C76019701B9
:108AB0008601B701A6010E94F5320F900F900F902A
:108AC0000F900F900E943B1D809151099091520987
:108AD000A0915309B09154090197A105B10561F521
:108AE0000E943B1D8091910990919209A091930958
:108AF000B09194090197A105B105F1F48BE297E0DB
:108B00000E9439160E946D2C1F921F9221E02F9314
:108B10001F921F92912C812CB12CA12CC12CD12CF5
:108B2000760197018601B701A6010E94F5320F90E8
:108B30000F900F900F900F9088E692E00E943916E8
:108B400086E692E00E94391683E497E00E94391687
:108B500083E692E00E943916EEE06E2E712CFEED57
:108B60002F2EF2E03F2E0E94640AAB01BC018091DF
:108B70002F0890913008A0913108B0913208481721
:108B800059076A077B0708F060C040932F0850938D
:108B90003008609331087093320881ED9CE00E94A8
:108BA000F707892B09F433C30E94640A60933E09D6
:108BB00070933F09809340099093410981ED9CE0B7
:108BC0000E94D50780932A09982F9F7D953409F438
:108BD00068C02091280930912909F901EC53F74F19
:108BE00080832F5F3F4F309329092093280980917C
:108BF0002809909129098336910564F02AE0209391
:108C00002A09FC01EC53F74F208301969093290920
:108C100080932809209128093091290980912A09F7
:108C20008A3021F0243631050CF4F1C2C9010197D4
:108C3000AFE5B8E0E4ECF8E0AF01445C5840481719
:108C40005907B4F541914D93F7CF481B590B6A0B67
:108C50007B0B483E53406105710508F49ECF885157
:108C60009C4FAF4FBF4F80932F0890933008A09335
:108C70003108B09332080E94341EEC010E94CB16DA
:108C8000CE010C960E94CB16CE0148960E94CB16C0
:108C9000CE0184960E94CB16CE01C0960E94CB16C0
:108CA0007CCF0E945D1421E0DC011E962C939FCFA7
:108CB000815A974FFC011082223031050CF4A3C277
:108CC0008AE593E00E94391682E194E00E94391609
:108CD0008CE597E00E9439168FE598E00E943916DE
:108CE0008CE597E00E9439168EED97E00E943916C8
:108CF0008AE390E00E943A4FEC011A821B821C82A8
:108D00001D821E821F82188619861A861B861C8663
:108D10001D861E861F86188A198A1A8A1B8A1C8A33
:108D20001D8A1E8A1F8A188E198E1A8E1B8E1C8E03
:108D30001D8E1E8E1F8E18A219A21AA21BA21CA283
:108D40001DA21EA21FA218A619A61AA61BA61CA623
:108D50001DA61EA61FA618AA19AA1AAA1BAA1CAAF3
:108D60001DAA1EAA1FAA18AE19AE6DE172E08FE50A
:108D700098E00E9462508C01DC018C918654823014
:108D800008F0EDC16EE577E0C8010E945358892BC9
:108D900009F49DC161E677E0C8010E945358892B10
:108DA00009F495C165E677E0C8010E945358892B04
:108DB00009F490C168E677E0C8010E945358892BF6
:108DC00009F488C16CE677E0C8010E945358892BEA
:108DD00009F483C160E777E0C8010E945358892BEA
:108DE00009F47EC164E777E0C8010E945358892BDB
:108DF00009F476C167E777E0C8010E945358892BD0
:108E000009F471C16BE777E0C8010E945358892BC0
:108E100009F46CC16FE777E0C8010E945358892BB1
:108E200009F467C163E877E0C8010E945358892BB1
:108E300009F462C167E877E0C8010E945358892BA2
:108E400009F45DC16BE877E0C8010E945358892B93
:108E500009F458C16FE877E0C8010E945358892B84
:108E600009F453C163E977E0C8010E945358892B84
:108E700009F44EC167E977E0C8010E945358892B75
:108E800009F449C16BE977E0C8010E945358892B66
:108E900009F444C16FE977E0C8010E945358892B57
:108EA00009F43FC163EA77E0C8010E945358892B57
:108EB00009F43AC167EA77E0C8010E945358892B48
:108EC00009F435C16BEA77E0C8010E945358892B39
:108ED00009F430C16FEA77E0C8010E945358892B2A
:108EE00009F42BC163EB77E0C8010E945358892B2A
:108EF00009F426C167EB77E0C8010E945358892B1B
:108F000009F421C16BEB77E0C8010E945358892B0B
:108F100009F41CC16FEB77E0C8010E945358892BFC
:108F200009F417C163EC77E0C8010E945358892BFC
:108F300009F012C188EB90E0909301028093000247
:108F40000115110509F411C1F8018081883541F43A
:108F5000C80101960E945F506A837B838C839D8346
:108F6000D8018C91893541F4C80101960E945F5067
:108F70006E837F8388879987F80180818A3541F4E1
:108F8000C80101960E945F506A877B878C879D8706
:108F9000D8018C91813451F4C80101960E945F5030
:108FA0000E940F576E877F87888B998BF80180818D
:108FB000823451F4C80101960E945F500E940F57FD
:108FC0006A8B7B8B8C8B9D8BD8018C91833451F475
:108FD000C80101960E945F500E940F576E8B7F8BD5
:108FE000888F998FF8018081833541F4C8010196FB
:108FF0000E945F506A8F7B8F8C8F9D8FD8018C91E0
:10900000803551F4C80101960E945F500E940F57AD
:109010006E8F7F8F88A399A3F8018081863551F4E4
:10902000C80101960E945F500E940F576AA37BA35C
:109030008CA39DA3D8018C91873551F4C80101966A
:109040000E945F500E940F576EA37FA388A799A725
:10905000F8018081853451F4C80101960E945F5067
:109060000E940F576AA77BA78CA79DA7D8018C9158
:10907000843551F4C80101960E945F500E940F5739
:109080006EA77FA788AB99ABF80180818D3451F42E
:10909000C80101960E945F500E940F576AAB7BABDC
:1090A0008CAB9DABD8018C91813551F4C8010196F0
:1090B0000E945F500E940F576EAB7FAB88AF99AF95
:1090C00067EC77E090E080E0FDD78C0139CF90E04D
:1090D00080E032CF81E090E02FCF8CE190E02CCF88
:1090E0008DE690E029CF8FE690E026CF80E790E0F4
:1090F00023CF81E790E020CF82E790E01DCF83E788
:1091000090E01ACF84E790E017CF88E790E014CF83
:1091100089E790E011CF8AE790E00ECF83E890E0F6
:109120000BCF84E890E008CF8DE890E005CF8EE883
:1091300090E002CF8FE890E0FFCE80E990E0FCCE97
:1091400081EA90E0F9CE85EB90E0F6CE86EB90E0F8
:10915000F3CE87EB90E0F0CE8FEF9FEFEDCE8FEF69
:109160009FEF90930102809300020E945D14FC0126
:1091700016850E943B1D80905D0990905E09A0902D
:109180005F09B0906009CEA8DFA8E8ACF9AC0E94F6
:109190005D14C092CD0CD092CE0CE092CF0CF09228
:1091A000D00C80910002909101028230910508F468
:1091B0009DC49C012F5631092530310508F496C411
:1091C000552453948437910509F0512C112309F447
:1091D00091C48D36910509F48DC49C01285731093D
:1091E0002330310508F486C4855B9109039708F4A0
:1091F00081C486E593E00E9439160E945D140E94A6
:109200003A16CE01D3D610922909109228098091DE
:109210002B098111A4C00E945D14FC01868588235E
:1092200009F49DC00E946D2CEC01FC01EE5DFC4F29
:10923000108240960E94BB0CCE018C569F4F0E941C
:10924000BB0CCE01885E9E4F0E94BB0C0E9448154D
:109250008C010F5F1F4FC1E0D0E0D8018D918D01CF
:109260008823D9F081E993E00E94391681EE97E0D6
:109270000E943916CE010E9434168EED97E00E94AE
:10928000391660E08C2F0E945C0970E060E0CE012E
:109290000E946916F80131971082F80187A9882386
:1092A000F9F081E993E00E94391688EF97E00E9477
:1092B0003916CE010E9434168EED97E00E943916C1
:1092C00061E08C2F0E94890960E08C2F0E945C096C
:1092D00061E070E0CE010E946916D801D7961C9219
:1092E0002196C533D10509F0B8CF0E94EE14209124
:1092F000FF0D30E0C901880F991F820F931FFC01F9
:10930000E259F24F80818F7B80832091020E30E002
:10931000C901880F991F820F931FFC01E259F24F78
:1093200080818F7B80832091050E30E0C901880FFA
:10933000991F820F931FFC01E259F24F80818F7BAE
:1093400080832091080E30E0C901880F991F820F99
:10935000931FFC01E259F24F80818F7B80830E9432
:109360005D14FC01868580932B090E943B1D209192
:109370002C0930912D09DC0112968D919C912817B2
:109380003907A9F00E943B1DFC01828193819093D3
:109390002D0980932C090E946D2C0E94C7280E94E1
:1093A0006D2C0E9481270E94341E0E94041E0E9480
:1093B000640A00913E0910913F09209140093091C3
:1093C0004109601771078207930708F0F0C20E94F5
:1093D000640A60933E0970933F098093400990931B
:1093E00041090E949D08BFCB209779F48EE493E059
:1093F0000E9439160E945D140E943A160E945D1464
:1094000070925E0860925D08FCCEE0900002F090E1
:109410000102FFEFEF16FF0649F3E114F10409F032
:1094200083C080915B0890915C08892B61F482E095
:1094300090E020D528E333E0DC012D933C9390931A
:109440005C0880935B0800915B0810915C08B1E7B1
:10945000EB16F10409F09EC08091510890915208DA
:10946000892B61F482E090E005D526E033E0FC0131
:1094700031832083909352088093510800915108C2
:1094800010915208F9E7EF16F10409F09EC080919F
:10949000470890914808892B61F482E090E0EAD473
:1094A000E4EDF2E0DC01ED93FC93909348088093A7
:1094B00047080091470810914808F0E9EF16F104B9
:1094C00009F09EC080913D0890913E08892B61F47F
:1094D00082E090E0CFD4E2EAF2E0DC01ED93FC938D
:1094E00090933E0880933D0800913D0810913E08FE
:1094F000F8EBEF16F10409F09EC0809133089091CB
:109500003408892B61F482E090E0B4D4E0E7F2E023
:10951000DC01ED93FC939093340880933308009121
:1095200033081091340887C0BCE1EB16F104B9F49C
:109530008091590890915A08892B61F482E090E05B
:1095400099D42EE233E0FC013183208390935A08B2
:10955000809359080091590810915A0878CFFDE678
:10956000EF16F10409F082C08091570890915808D5
:10957000892B61F482E090E07DD424E233E0DC01C9
:109580002D933C9390935808809357080091570867
:1095900010915808F2E7EF16F10409F082C08091AB
:1095A0004F0890915008892B61F482E090E062D4DA
:1095B0002CEF32E0DC012D933C9390935008809384
:1095C0004F0800914F0810915008FAE7EF16F10488
:1095D00009F082C08091450890914608892B61F47A
:1095E00082E090E047D4EAECF2E0DC01ED93FC93FA
:1095F00090934608809345080091450810914608CD
:10960000F1EAEF16F10409F082C080913B089091D5
:109610003C08892B61F482E090E02CD4E8E9F2E088
:10962000DC01ED93FC9390933C0880933B08009100
:109630003B0810913C080115110509F044C18EE466
:1096400093E00E9439160E945D140E943A160E940F
:109650005D1470925E0860925D088BEC97E00E944A
:10966000BC158EED97E00E94BC15CBCDBFE6EB1686
:10967000F10409F068C08091550890915608892B33
:1096800061F482E090E0F6D32AE133E0FC0131831B
:1096900020839093560880935508009155081091A7
:1096A0005608B3E7EB16F10409F0BBC080914D08F2
:1096B00090914E08892B61F482E090E0DBD322EF99
:1096C00032E0FC013183208390934E0880934D0853
:1096D00000914D0810914E08FDE8EF16F10409F0D5
:1096E000BBC08091430890914408892B61F482E0CB
:1096F00090E0C0D3E0ECF2E0DC01ED93FC939093BA
:109700004408809343080091430810914408F5EB06
:10971000EF16F10409F0BBC08091390890913A0826
:10972000892B61F482E090E0A5D3EEE8F2E0DC0161
:10973000ED93FC9390933A0880933908009139088F
:1097400010913A0878CFF0E7EF16F10409F066C0FF
:109750008091530890915408892B61F482E090E045
:1097600089D320E133E0DC012D933C93909354089E
:10977000809353080091530810915408B8E7EB16F2
:10978000F10409F07FCE8091490890914A08892B15
:1097900051F482E090E06ED3FC01318220829093FC
:1097A0004A08809349080091490810914A08FFE847
:1097B000EF16F10409F081CE80913F0890914008A6
:1097C000892B61F482E090E055D3ECEAF2E0DC0111
:1097D000ED93FC939093400880933F0800913F08DD
:1097E00010914008F7EBEF16F10409F081CE80915B
:1097F000350890913608892B61F482E090E03AD3E5
:10980000EAE7F2E0DC01ED93FC9390933608809355
:10981000350800913508109136080DCF10E000E0B2
:1098200016CEF4E7EF16F10409F0A8CF80914B08AB
:1098300090914C08892B61F482E090E01BD328EED4
:1098400032E0DC012D933C9390934C0880934B08BD
:1098500000914B0810914C08FEE8EF16F10409F056
:10986000A6CF8091410890914208892B61F482E053
:1098700090E000D3E6EBF2E0DC01ED93FC939093F3
:109880004208809341080091410810914208F6EB8C
:10989000EF16F10409F0A6CF8091370890913808AF
:1098A000892B61F482E090E0E5D2E4E8F2E0DC01AB
:1098B000ED93FC9390933808809337080091370814
:1098C00010913808B8CE8AE493E00E9439160E94BD
:1098D0005D140E943A160E945D1410925E08109268
:1098E0005D08F12CE12C2FEFE21AF20A31E0E316C9
:1098F000F10441F086E493E00E9439160E945D1461
:109900000E943A16D801ED91FC910480F581E02D7A
:10991000BE01C80119950E945D14C0905D08D090E9
:109920005E080E945D14FC01868581110AC0E8145E
:10993000F9043CF4C114D10421F0F2E0CF16D104B3
:1099400091F681ED9CE00E94F707181619062CF499
:1099500081ED9CE00E94D507F4CFCD2809F4B3C077
:109960005520A1F00E943B1D8091590990915A0900
:10997000A0915B09B0915C090197A105B10531F493
:109980000E945D1421E0DC011E962C938EE393E08F
:109990000E9439168EE098E00E9439160E945D14EC
:1099A00080915D0890915E080E94341690C0601B03
:1099B000710B820B930B693873418105910508F493
:1099C00010CD0E945D14DC011E968C91882309F451
:1099D00077C086E693E00E9439160E945D140E94CB
:1099E0003A160E946D2CEC010E945D14FE01EC5AA7
:1099F000FF4F80819181A281B38180932E09909342
:109A00002F09A0933009B09331090E945D14FE0123
:109A1000E852FF4F80819181A281B3818093320906
:109A200090933309A0933409B09335090E945D14D3
:109A3000C45ADE4F88819981AA81BB8180933609FF
:109A400090933709A0933809B09339090E945D14A7
:109A50000E94261B0E946D2C0E94C61B0E945D1452
:109A60000E94A9140E945D140E94A8190E943B1D27
:109A70008091510990915209A0915309B0915409D4
:109A80000197A105B10541F08EE593E00E943916DA
:109A90000E945D140E943A1680913A0990913B0908
:109AA000A0913C09B0913D090196A11DB11D809383
:109AB0003A0990933B09A0933C09B0933D0987CCA8
:109AC00082E693E088CF82E493E00E9439160E94F8
:109AD0005D140E943A160E945D141092CD0C1092F3
:109AE000CE0C1092CF0C1092D00C8BCB55245394EB
:109AF00011117FCB0E943B1D809151099091520919
:109B0000A0915309B09154090197A105B10509F439
:109B10006BCC552009F468CC82E593E00E9439169D
:109B20000E945D140E943A160E945D148FE090E03E
:109B300090935E0880935D0864CB87E49EE00E946A
:109B4000B12987E39EE00E94B12987E29EE00E944E
:109B5000B12987E19EE00E94B12987E89EE00E943A
:109B6000B12987E79EE00E94B12987E69EE00E9426
:109B7000B12987E59EE00E94B12987EC9EE00E9412
:109B8000B12987EB9EE00E94B12987EA9EE00E94FE
:109B9000B12987E99EE00E94B12987E09FE00E94F9
:109BA000B12987EF9EE00E94B12987EE9EE00E94D6
:109BB000B12987ED9EE00E94B12987E49FE00E94D1
:109BC000B12987E39FE00E94B12987E29FE00E94CC
:109BD000B12987E19FE00E94B12987E89FE00E94B8
:109BE000B12987E79FE00E94B12987E69FE00E94A4
:109BF000B12987E59FE00E94B12987EC9FE00E9490
:109C0000B12987EB9FE00E94B12987EA9FE00E947B
:109C1000B12987E99FE00E94B12987E090E10E9485
:109C2000B12987EF9FE00E94B12987EE9FE00E9453
:109C3000B12987ED9FE00E94B12987E490E10E945D
:109C4000B12987E390E10E94B12987E290E10E9467
:109C5000B12987E190E10E94B12987E890E10E9453
:109C6000B12987E790E10E94B12987E690E10E943F
:109C7000B12987E590E10E94B12987EC90E10E942B
:109C8000B12987EB90E10E94B12987EA90E10E9417
:109C9000B12987E990E10E94B12987E091E10E9412
:109CA000B12987EF90E10E94B12987EE90E10E94EF
:109CB000B12987ED90E10E94B12987E491E10E94EA
:109CC000B12987E391E10E94B12987E291E10E94E5
:109CD000B12987E191E10E94B12987E891E10E94D1
:109CE000B12987E791E10E94B12987E691E10E94BD
:109CF000B12987E591E10E94B12987EC91E10E94A9
:109D0000B12987EB91E10E94B12987EA91E10E9494
:109D1000B12987E991E10E94B12987E092E10E948F
:109D2000B12987EF91E10E94B12987EE91E10E946C
:109D3000B12987ED91E10E94B12987E492E10E9467
:109D4000B12987E392E10E94B12987E292E10E9462
:109D5000B12987E192E10E94B12987E892E10E944E
:109D6000B12987E792E10E94B12987E692E10E943A
:109D7000B12987E592E10E94B12987EC92E10E9426
:109D8000B12987EB92E10E94B12987EA92E10E9412
:109D9000B12987E992E10E94B12987E093E10E940D
:109DA000B12987EF92E10E94B12987EE92E10E94EA
:109DB000B12987ED92E10E94B12987E493E10E94E5
:109DC000B12987E393E10E94B12987E293E10E94E0
:109DD000B12987E193E10E94B12987E893E10E94CC
:109DE000B12987E793E10E94B12987E693E10E94B8
:109DF000B12987E593E10E94B12987EC93E10E94A4
:109E0000B12987EB93E10E94B12987EA93E10E948F
:109E1000B12987E993E10E94B12987E094E10E948A
:109E2000B12987EF93E10E94B12987EE93E10E9467
:109E3000B12987ED93E10C94B129EF920F931F9311
:109E4000CF93DF93E80134E047FD34E1042E000CAA
:109E5000550B57FF03C0519541955109E32E022F31
:109E6000242FAE01ABD1CE01DF91CF911F910F9185
:109E7000EF9008950F931F93CF93DF938230910556
:109E800010F482E090E0E0911114F091121430E0AF
:109E900020E0B0E0A0E0309799F42115310509F4F5
:109EA0004AC0281B390B24303105D8F58A819B81A3
:109EB0006115710589F1FB0193838283FE0111C055
:109EC000408151810281138148175907E0F04817FA
:109ED000590799F4109761F012960C931297139604
:109EE0001C933296CF01DF91CF911F910F9108956E
:109EF0000093111410931214F4CF2115310551F071
:109F00004217530738F0A901DB019A01BD01DF01B7
:109F1000F801C1CFEF01F9CF90931214809311147F
:109F2000CDCFFE01E20FF31F8193919322503109AF
:109F300039832883D7CF20910F1430911014232B0D
:109F400041F42091040230910502309310142093C3
:109F50000F1420910202309103022115310541F4C2
:109F60002DB73EB74091060250910702241B350BD6
:109F7000E0910F14F0911014E217F307A0F42E1BD8
:109F80003F0B2817390778F0AC014E5F5F4F24175D
:109F9000350748F04E0F5F1F5093101440930F1475
:109FA000819391939FCFF0E0E0E09CCFCF93DF933C
:109FB0000097E9F0FC01329713821282A0911114EC
:109FC000B0911214ED0130E020E01097A1F420814F
:109FD0003181820F931F20910F1430911014281794
:109FE000390709F061C0F0931014E0930F14DF916A
:109FF000CF910895EA01CE17DF07E8F54A815B812A
:10A000009E0141155105B1F7E901FB83EA834991AE
:10A010005991C40FD51FEC17FD0761F48081918120
:10A020000296840F951FE901998388838281938129
:10A030009B838A83F0E0E0E012968D919C911397C8
:10A040000097B9F52D913C911197CD010296820FA1
:10A05000931F20910F14309110142817390739F6E7
:10A06000309751F51092121410921114B0931014ED
:10A07000A0930F14BCCFD383C28340815181840F3E
:10A08000951FC817D90761F44E5F5F4F888199818A
:10A09000480F591F518340838A819B819383828318
:10A0A0002115310509F0B0CFF0931214E09311148B
:10A0B0009ECFFD01DC01C0CF13821282D7CF66276D
:10A0C0007727F4C14DE054E100C0FA01A191B081BD
:10A0D000009719F41097E1F0CD01DC01CD010D904E
:10A0E000002011F4C00113C0FB012191222319F0BB
:10A0F0002015D9F7F3CFFB012191201519F41E92F9
:10A10000119606C02223C1F70D900020A1F7D001BF
:10A11000FA01A193B0830895BB274A3031F4992303
:10A1200022F4BDE2909581959F4F30C0BB272A3025
:10A1300051F4992342F4BDE2909580957095619514
:10A140007F4F8F4F9F4F01C0BB27FA01A62F621789
:10A15000710581059105330B30FB66F0AA27660F68
:10A16000771F881F991FAA1FA21710F0A21B6395C3
:10A170003850A9F7A05DAA3308F0A95DA19336F77E
:10A18000B111B1931082CA01DEC3BB27FB01552771
:10A19000AA27880F991FAA1FA41710F0A41B839544
:10A1A0005051B9F7A05DAA3308F0A95DA1930097BB
:10A1B00079F7B111B1931192CB01C5C38F929F92E0
:10A1C000AF92BF92CF92DF92EF92FF920F931F93C5
:10A1D000CF93DF9300D000D000D0CDB7DEB76A01B7
:10A1E000F22EB02E102FFBE3AF2EA01608F41BE3C7
:10A1F0001F5F012F27E0AE014F5F5F4FACD2BC0164
:10A200008981982F9970913009F44EC09BE2E1FC4E
:10A2100004C09E2D9170E0FC49C05E2D5071E82F66
:10A22000E87083FF55C084E0911101C083E0EF2DF9
:10A23000E81B8F1508F0E0E0D6018E2F20E25523B1
:10A24000C9F1992329F0D6019C93C60101966C01AE
:10A2500096012D5F3F4FE2FE33C08EE4D6018C9312
:10A2600091E411969C93119712968C93D9018E2F9D
:10A2700090E281112AC0E20FF32FF11D10828EEFC0
:10A280009FEF29960FB6F894DEBF0FBECDBFDF91CA
:10A29000CF911F910F91FF90EF90DF90CF90BF90E3
:10A2A000AF909F908F9008959DE2B7CF90E2B5CF89
:10A2B0002D9381508111FCCFCE0ED11CE0E0C1CF97
:10A2C0008EE6D6018C9391E6CCCF9D938150D1CF71
:10A2D000482F447082FF3DC084E0911101C083E0AB
:10A2E0008F1510F4EF2DE81BD6018E2F20E2552399
:10A2F00009F1992329F0D6019C93C60101966C01BE
:10A3000096012D5F3F4FE2FE1BC089E4D6018C937E
:10A310008EE411968C93119786E412968C93D90152
:10A320008E2F90E2882309F4A6CF9D938150FACF17
:10A330002D9381508111FCCFCE0ED11CE0E0D9CFFE
:10A3400089E6D6018C938EE611968C93119786E65A
:10A35000E4CF9B0177FF02C030E020E0A1E0B0E055
:10A36000911102C0B0E0A0E0F9013196AE0FBF1F1D
:10A370008B2C912CBB2009F461C05401EFEFAE1A75
:10A38000BE0AAA0DBB1DFA161B0619F014F04F2DBC
:10A390004A1B511188C0E3FC59C07601A42FB0E2DA
:10A3A000A1114FC0C40ED11C992309F45BC040E039
:10A3B000D6011196F60190836D01552309F448C02A
:10A3C000012F060F9A81582F507184FF03C09133DB
:10A3D00009F4015010160CF047C0093008F008E0ED
:10A3E000EEE2FE2E5B01A01AB108850191948194E2
:10A3F00091082F3F320729F4D601FC92F6013196DD
:10A400006F016217730794F1021713077CF5DB01E4
:10A41000A21BB30BAA24A394B12CAC0EBD1EAA0D93
:10A42000BB1D11968C9121503109D601119628152A
:10A430003905F4F0F60180836D01DBCFB12CA12C3E
:10A44000A0CFF701B1937F01A150AACF9111B0CF56
:10A45000D601942F50E302C05D9391509111FCCF2F
:10A46000C40ED11C40E0ACCF01E0BACF80E3DBCF1B
:10A470006217730731F4963388F4953311F455233A
:10A4800069F0F6018083FD01842F90E2811108C0FC
:10A49000A40FB11D1C9290E080E0F3CE81E3F1CFD8
:10A4A00091938150F3CF911183CF8ACF8F929F9256
:10A4B000AF92BF92CF92DF92EF92FF920F931F93D2
:10A4C000CF93DF935C017B016115710519F0DB010E
:10A4D0008D939C9385010F5F1F4FF501D0818D2FC8
:10A4E00090E011D26C01892BA9F5DD32A9F50F5F3F
:10A4F0001F4FD5011196DC91C1E05801F1E0AF1A70
:10A50000B10843E050E06CEE70E0C50104D2892B45
:10A5100061F5680182E0C80ED11C45E050E067EEAD
:10A5200070E0C601F8D1892B21F4680197E0C90ECB
:10A53000D11CE114F10419F0D701CD92DC9260E056
:10A5400070E080E89FEFC111F9C060E070E080E842
:10A550009FE7F4C05801BECFDB3229F485010E5FBE
:10A560001F4FF501D181C0E0C8CF43E050E064EE59
:10A5700070E0C501D0D1892BE9F0F80110E000E0CE
:10A5800020E030E0A9015F01B0ED8B2E8D0E89E057
:10A590008815C0F19C2E689491F88C2F8870C2FFAA
:10A5A00016C0811102C00F5F1F4F3196D501DC919B
:10A5B000C92DE9CFE114F10429F00E5F1F4FF70117
:10A5C0001183008360E070E080EC9FE7B7C08823D0
:10A5D00011F001501109A5E0B0E013D39B01AC01CB
:10A5E000220F331F441F551F280D311D411D511DC2
:10A5F000283999E93907490799E15907B0F2C66046
:10A600009C2ED3CFAEEF8A1206C0C3FD3CC09C2E59
:10A61000689493F8CACFDF7DD534A9F580818D3257
:10A6200039F4C061DF011296818162E070E006C0FA
:10A63000DF018B32C1F3119661E070E080535D0160
:10A64000A61AB70A8A30F8F4E0E8CE16ECE0DE0687
:10A650005CF4B601660F771F660F771FC60ED71E14
:10A66000CC0CDD1CC80ED11C5D01FFEFAF1ABF0A78
:10A670008C9180538A3098F1C4FF03C0D194C19467
:10A68000D1080C0D1D1DC1FF09C0E114F10431F00A
:10A6900081E0A81AB108D701AD92BC92CA01B901F4
:10A6A00066D1C370C33009F490584B015C0120E0BF
:10A6B00030E0A90158D1882309F43EC0CBE1D1E0B4
:10A6C00017FF05C0119501951109C3E0D1E06E0196
:10A6D000B8E1CB1AD10880E2E82EF12C0EC0D501EA
:10A6E000B3CFFE0125913591459154910E191F0963
:10A6F000C501B4019DD14B015C01D501C4010E150A
:10A700001F057CF72497F594E794CC16DD06A9F78E
:10A710008A2F880F8B2F881F8F3F41F020E030E079
:10A72000A901C501B4011FD1811106C082E290E0E8
:10A730009093141480931314C501B401DF91CF9149
:10A740001F910F91FF90EF90DF90CF90BF90AF904F
:10A750009F908F900895283008F027E03327DA0182
:10A76000990F311D87FD916000966105710539F4DF
:10A7700032602E5F3D9330E32A95E1F708959F3FC5
:10A7800030F080387105610509F03C5F3C5F3D9316
:10A79000913008F08068911DDF93CF931F930F9342
:10A7A000FF92EF92192F987F9695E92F969596959F
:10A7B000E90FFF27E758FE4F99273327EE24FF24A0
:10A7C000A701E70105900894079428F4360FE71EC7
:10A7D000F81E491F511D660F771F881F991F069489
:10A7E000A1F70590079428F4E70EF81E491F561F9D
:10A7F000C11D770F881F991F661F0694A1F705904A
:10A80000079428F4F80E491F561FC71FD11D880F43
:10A81000991F661F771F0694A1F70590079420F4EF
:10A82000490F561FC71FD81F990F661F771F881F14
:10A830000694A9F784911095177041F0D695C795A5
:10A8400057954795F794E7941A95C1F7EFE1F1E032
:10A8500068941590159135916591959105907FE2D9
:10A860007395E118F10A430B560BC90BD009C0F7D9
:10A87000E10CF11E431F561FC91FD01D7EF470331B
:10A8800011F48A95E6CFE894015030F0080F0AF4ED
:10A890000027021708F4202F2395022F7A3328F07F
:10A8A00079E37D932A95E9F710C07D932A9589F67F
:10A8B000069497956795379517951794E118F10ABF
:10A8C000430B560BC90BD00998F023957E917395D5
:10A8D0007A3308F070E37C932013B8F77E917061AF
:10A8E0007D9330F0839571E37D9370E32A95E1F7D2
:10A8F0001124EF90FF900F911F91CF91DF91992735
:10A9000087FD909508959111F6C0803219F0895015
:10A910008550D0F70895FB01DC014150504088F08C
:10A920008D9181341CF08B350CF4805E659161341F
:10A930001CF06B350CF4605E861B611171F3990B92
:10A940000895881BFCCFDC01FC01672F71917723F0
:10A95000E1F7329704C07C916D9370836291AE17DA
:10A96000BF07C8F3089540D008F481E00895E89443
:10A9700009C097FB3EF490958095709561957F4F47
:10A980008F4F9F4F9923A9F0F92F96E9BB279395F5
:10A99000F695879577956795B795F111F8CFFAF405
:10A9A000BB0F11F460FF1BC06F5F7F4F8F4F9F4F36
:10A9B00016C0882311F096E911C0772321F09EE894
:10A9C000872F762F05C0662371F096E8862F70E0FA
:10A9D00060E02AF09A95660F771F881FDAF7880FD4
:10A9E0009695879597F90895990F0008550FAA0B2A
:10A9F000E0E8FEEF16161706E807F907C0F0121692
:10AA00001306E407F50798F0621B730B840B950B94
:10AA100039F40A2661F0232B242B252B21F40895E9
:10AA20000A2609F4A140A6958FEF811D811D089586
:10AA30000BD07BC06CD028F071D018F0952309F0B2
:10AA40005DC062C01124A5C081D0A0F3959FD1F351
:10AA5000950F50E0551F629FF001729FBB27F00DCC
:10AA6000B11D639FAA27F00DB11DAA1F649F662721
:10AA7000B00DA11D661F829F2227B00DA11D621F70
:10AA8000739FB00DA11D621F839FA00D611D221F2A
:10AA9000749F3327A00D611D231F849F600D211D0E
:10AAA000822F762F6A2F11249F5750408AF0E1F0B1
:10AAB00088234AF0EE0FFF1FBB1F661F771F881FFA
:10AAC00091505040A9F79E3F510570F017C061C0EA
:10AAD0005F3FECF3983EDCF3869577956795B795E5
:10AAE000F795E7959F5FC1F7FE2B880F911D96950F
:10AAF000879597F9089599278827089597F99F676B
:10AB000080E870E060E008959FEF80EC08950024F5
:10AB10000A941616170618060906089500240A94C2
:10AB200012161306140605060895092E0394000C48
:10AB300011F4882352F0BB0F40F4BF2B11F460FFD7
:10AB400004C06F5F7F4F8F4F9F4F089557FD905800
:10AB5000440F551F59F05F3F71F04795880F97FBE1
:10AB6000991F61F09F3F79F087950895121613069B
:10AB70001406551FF2CF4695F1DF08C016161706CA
:10AB80001806991FF1CF86957105610508940895FF
:10AB9000E894BB2766277727CB0197F90895F999A1
:10ABA000FECF92BD81BDF89A992780B50895262FD2
:10ABB000F999FECF1FBA92BD81BD20BD0FB6F894A2
:10ABC000FA9AF99A0FBE01960895052E97FB16F48E
:10ABD00000940FD057FD05D024D007FC02D046F4D6
:10ABE00008C050954095309521953F4F4F4F5F4F8E
:10ABF000089590958095709561957F4F8F4F9F4FE9
:10AC0000089531D0A59F900DB49F900DA49F800D05
:10AC1000911D11240895B7FFF4CFF3DF821B930B2E
:10AC20000895A1E21A2EAA1BBB1BFD010DC0AA1F8D
:10AC3000BB1FEE1FFF1FA217B307E407F50720F0A5
:10AC4000A21BB30BE40BF50B661F771F881F991F20
:10AC50001A9469F760957095809590959B01AC0169
:10AC6000BD01CF010895A29FB001B39FC001A39F72
:10AC7000700D811D1124911DB29F700D811D112435
:10AC8000911D08955058BB27AA270ED04ECF3FDF05
:10AC900030F044DF20F031F49F3F11F41EF434CF44
:10ACA0000EF4E095E7FB2ACFE92F50DF80F3BA17C7
:10ACB000620773078407950718F071F49EF568CF53
:10ACC0000EF4E0950B2EBA2FA02D0B01B9019001C7
:10ACD0000C01CA01A0011124FF27591B99F0593F0B
:10ACE00050F4503E68F11A16F040A22F232F342F53
:10ACF0004427585FF3CF469537952795A795F040A1
:10AD00005395C9F77EF41F16BA0B620B730B840BB5
:10AD1000BAF09150A1F0FF0FBB1F661F771F881F6D
:10AD2000C2F70EC0BA0F621F731F841F48F48795C5
:10AD300077956795B795F7959E3F08F0B3CF9395B4
:10AD4000880F08F09927EE0F9795879508950CD0F6
:10AD5000ECCEE4DE40F0DBDE30F021F45F3F19F0B2
:10AD6000CDCE511116CFD0CEF1DE98F39923C9F391
:10AD70005523B1F3951B550BBB27AA276217730701
:10AD8000840738F09F5F5F4F220F331F441FAA1FB5
:10AD9000A9F333D00E2E3AF0E0E830D09150504075
:10ADA000E695001CCAF729D0FE2F27D0660F771F23
:10ADB000881FBB1F261737074807AB07B0E809F005
:10ADC000BB0B802DBF01FF2793585F4F2AF09E3F9A
:10ADD000510568F093CEDDCE5F3FECF3983EDCF397
:10ADE000869577956795B795F7959F5FC9F7880F13
:10ADF000911D9695879597F90895E1E0660F771F65
:10AE0000881FBB1F621773078407BA0720F0621BF5
:10AE1000730B840BBA0BEE1F88F7E095089504D0EE
:10AE20006894B111B6CE089599DE88F09F5790F0DE
:10AE3000B92F9927B751A0F0D1F0660F771F881F5F
:10AE4000991F1AF0BA95C9F712C0B13081F0A0DE8F
:10AE5000B1E008959DCE672F782F8827B85F39F02D
:10AE6000B93FCCF3869577956795B395D9F73EF4BE
:10AE700090958095709561957F4F8F4F9F4F089566
:10AE8000B3DD08F48FEF0895AFDD880B990B0895BB
:10AE9000DB018F939F93B5DEBF91AF91A29F800D91
:10AEA000911DA39F900DB29F900D11240895991BA1
:10AEB00079E004C0991F961708F0961B881F7A95B1
:10AEC000C9F780950895EE0FFF1F881F8BBF07906D
:10AED000F691E02D19944F925F926F927F928F922C
:10AEE0009F92AF92BF92CF92DF92EF92FF920F9319
:10AEF0001F93CF93DF938C01009799F4CB01DF91DF
:10AF0000CF911F910F91FF90EF90DF90CF90BF9066
:10AF1000AF909F908F907F906F905F904F900C9428
:10AF20003A4FFC01E60FF71F9C0122503109E2174E
:10AF3000F30708F4ACC0D901CD91DC911197C61785
:10AF4000D70718F1C530D10570F0CE0104978617E8
:10AF5000970748F0C61BD70B2297C193D1936D93E7
:10AF60007C93CF0123D8C801DF91CF911F910F911E
:10AF7000FF90EF90DF90CF90BF90AF909F908F9019
:10AF80007F906F905F904F9008955B01AC1ABD0A5F
:10AF90004C018C0E9D1EA0911114B0911214512CD5
:10AFA000412CF12CE12C109731F580910F149091E8
:10AFB00010148815990509F05CC04616570608F06C
:10AFC00058C08091020290910302009741F48DB71E
:10AFD0009EB74091060250910702841B950BE8171B
:10AFE000F90708F054C0F0931014E0930F14F9011E
:10AFF00071836083B8CF8D919C91119712966C905C
:10B00000129713967C901397A815B90559F56C0102
:10B0100042E0C40ED11CCA14DB0420F1AC014A1971
:10B020005B09DA011296159780F062827382518370
:10B030004083D9016D937C93E114F10471F0D70141
:10B040001396FC93EE9312978ECF22968C0F9D1F32
:10B05000F90191838083F301EFCFF0931214E09311
:10B06000111481CF4816590608F42C017D01D30133
:10B070009ACFCB010E943A4F7C01009741F0AE017C
:10B08000B80108D0C8010E94D64F87016CCF10E0EC
:10B0900000E069CFFB01DC0102C001900D9241503C
:10B0A0005040D8F70895FB01DC018D910190801983
:10B0B0000110D9F3990B0895FB01DC0101900D9269
:10B0C0000020E1F7089511E0CEE9D1E000E005C0ED
:10B0D000802FFE01F8DE2196011DCF39D10780E0D7
:08B0E0000807B1F7F894FFCF57
:10B0E800FFFF000015148000362E352E302E450047
:10B0F80000010000000100000001000000200A0D0E
:10B108000000523835005238340052303500523180
:10B118003300523132005231310052373300523746
:10B128003200523731005231370052313600523135
:10B13800350052303400523837000D0A00200052D2
:10B148003939000D0A00200052393900000000008A
:10B158001B13D529A32C000000005914DF29461A17
:10B1680000000000800FCB29C11B0000000019134C
:10B17800D129D219000000007B0FC5290115000054
:10B1880000002C14DB297215000000001813CF29C9
:10B198006515000000007A0FC3291217000000008F
:10B1A8005C14E529AC15000000005814DD29572966
:10B1B800000000005B14E329A329000000002C0C08
:10B1C800BB29AE1D000000002D0CB9292C3B000046
:10B1D80000005A14E129433E000000001814D72942
:10B1E8000A3E000000001A13D329643D0000000045
:10B1F8002E0CBD29653B000000007F0FC9299C3C2F
:10B2080000000000790FC129E814000000002F0C8D
:10B21800BF29F13B000000001713CD29283D52300B
:10B228003300523032005230370052303100523041
:10B238003900523838005238370052303800523806
:10B248003800523030005238370052303600000093
:10B2580000002E089907C6077E08F707D507E907F3
:10B26800000000002B0CD929205100523431005025
:10B2780000523939002073746120002063757220F0
:10B288000020656E6420002068616C662000206CD8
:10B29800656E2000206D696E2000206D61782000A9
:10B2A8002073706420005238310020584100205823
:10B2B80042002059410020594200205A4100205A9A
:10B2C8004200686F6D650D0A0052323100523939FB
:10B2D800204572726F723A20696E76616C696420DB
:10B2E800706172616D657465722069640D0A00523F
:10B2F800383320006E616E00696E66006F766600F6
:10B3080052383200523230005239392057696C6C49
:10B31800207A65726F2058005239392057696C6C51
:10B32800207A65726F2059005239392057696C6C40
:10B33800207A65726F205A005239392043616C694E
:10B3480062726174696F6E206572726F723A2065FD
:10B358006E642073746F702061637469766520620F
:10B3680065666F72652073746172740D0A002061DE
:10B378007869732000206D6F766520746F20737470
:10B3880061727420666F722063616C6962726174A5
:10B39800696F6E0052393920656D657267656E6335
:10B3A800792073746F700D0A00523939206D6F76E9
:10B3B800656D656E7420646F6E650D0A002061749A
:10B3C800207374617274696E6720706F696E74009F
:10B3D800523233002063616C6962726174696E670E
:10B3E800206C656E67746800207374657020636FE5
:10B3F800756E743A200020617420656E6420706F49
:10B40800696E74002064656163746976617465208F
:10B418006D6F746F7220582064756520746F206D8D
:10B428006973736564207374657073002064656163
:10B4380063746976617465206D6F746F722059202A
:10B4480064756520746F206D697373656420737407
:10B458006570730020646561637469766174652042
:10B468006D6F746F72205A2064756520746F206D3B
:10B478006973736564207374657073005239392079
:10B4880074696D656F7574205820617869730D0A49
:10B49800005239392074696D656F757420592061BF
:10B4A8007869730D0A005239392074696D656F75B2
:10B4B80074205A20617869730D0A00523939206561
:10B4C80072726F720D0A005238390052393920737E
:10B4D800746F707065640D0A005239392065727294
:10B4E8006F72200053657269616C20636F6E6E65C0
:10B4F8006374696F6E207374617274656400536558
:10B508007420696E7075742F6F7574707574206609
:10B5180061726D626F742065787072657373005222
:10B5280065616420706172616D6574657273004C49
:10B538006F616420544D43206472697665727300AC
:10B54800496E697420544D43323133302064726936
:10B5580076657273004C6F616420544D4332313309
:10B568003020706172616D6574657273004C6F6133
:10B5780064206D6F76656D656E742073657474698B
:10B588006E677300536574206D6F746F7220656EFB
:10B5980061626C6573206F66660053746172742013
:10B5A80070696E20677561726400537461727420EB
:10B5B800736572766F00537461727420696E746576
:10B5C800727275707400436865636B20686F6D698B
:10B5D8006E67206F6E20626F6F7400523939204891
:10B5E8004F4D45205A204F4E2053544152545550E8
:10B5F8000D0A0052393920484F4D452059204F4EE9
:10B6080020535441525455500D0A0052393920489C
:10B618004F4D452058204F4E2053544152545550B9
:10B628000D0A0041524455494E4F2053544152543B
:10B63800555020434F4D504C455445002A00473043
:10B64800004730300047310047303100473238007A
:10B65800463039004639004631310046313200461D
:10B668003133004631340046313500463136004624
:10B67800323000463231004632320046333100461D
:10B688003332004634310046343200463433004603
:10B6980034340046363100463831004638320046E8
:10B6A80038330046383400200A0D005239392068F2
:10B6B800616E646C6572203D3D204E554C4C0D0A00
:10B6C8000020726573657474696E672064696769C0
:10B6D80074616C2070696E0020726573657474699A
:10B6E8006E6720616E616C6F672070696E0020560E
:02B6F800000050
:00000001FF
